:020000040000FA
:060000000DEF47F01200B5
:020006001200E6
:0600080058EF3BF012006E
:02000E001200DE
:020010000100ED
:0500120000000000F6F3
:06001800BBEF18F012001E
:02001E000800D8
:10002000AE8F0000FB070000040000006E8F000090
:100030009D0900004000000012000000FB060000C7
:1000400005000000458F0000C807000029000000DF
:10005000128F0000C806000033000000DC8E000094
:10006000C8050000360000007F8E00000009000077
:100070005D00000010000000FE040000020000000F
:10008000FAEC0CF040EC0DF0EE6AEE6AEE6AEE6A05
:1000900073EC0CF0EE6AEE6AEE6AEE6AAFEC09F011
:1000A000010EEE6E230EEE6E450EEE6E670EEE6ED8
:1000B000AFEC09F0040EF1EC0AF0890EEE6EAB0E17
:1000C000EE6ECD0EEE6EEF0EEE6EAFEC09F0080E9A
:1000D000F1EC0AF0FE0EEE6EDC0EEE6EBA0EEE6E77
:1000E000980EEE6EAFEC09F00C0EF1EC0AF0760E05
:1000F000EE6E540EEE6E320EEE6E100EEE6EE55299
:10010000E7CFD9FF1200FAEC0CF0080EE126030E3F
:10011000046E73EC0CF025EC0BF003E045EC0BF0F7
:10012000FDE13F0E00167FEC0BF0B4EC0CF0F90E85
:10013000DBCF04F0FA0EDBCF05F0066A076A05AEE6
:1001400002D006680768030E1F0B07E0D89004363C
:10015000053606360736E806F9E173EC0CF0045074
:10016000EF26EECF00F00550EF22EECF01F0065063
:10017000EF22EECF02F00750EF22EECF03F0F90EA0
:10018000DBCF08F0FA0EDBCF09F00A6A0B6A09AE82
:1001900002D00A680B68030E1F0B03E056EC0BF04D
:1001A000FDE10850005C095001580A5002580B50FC
:1001B000035806E240EC0DF0EE2AEE22EE22EE228B
:1001C0005DEC0BF0026A036A01AE02D002680368BC
:1001D0001D0E45EC0BF0FDE140EC0DF0EDEC0CF0EC
:1001E000400E046E056A066A076AD9CFE9FF2BEC58
:1001F0000BF0EE500758060E00C0DBFF070E01C0E3
:10020000DBFF5DEC0BF017EC0DF001500318E8AECE
:1002100002D0033404D00250005C035001586AE35A
:10022000060EDBCFE6FF070EDBCFE6FF19EC0BF087
:10023000F6EC0CF0E9CF02F0EACF03F0DB50E92452
:10024000006E010EDB50EA2075EC0BF0B5EC39F0D6
:10025000046E060EE15E0450F6EC0CF010EC0BF0B0
:10026000AFEC09F0E9CF02F0EACF03F034EC0BF089
:10027000060EDBCF28F0070EDBCF29F0040E28C0D6
:10028000DBFF050E29C0DBFF3F0EE76EDDEC0CF057
:10029000E7500026000E0122D6EC0CF001500318A6
:1002A000E8AE02D0033404D00250005C0350015881
:1002B0001EE2040EDBCF02F0050EDBCF03F0FB0ED7
:1002C000DB500224006EFC0EDB50032075EC0BF0BB
:1002D000AFEC09F0E9CF04F0EACF05F034EC0BF015
:1002E00033EC0DF0400EEE26000EED22CDD71EECC5
:1002F0000DF004D0040EDB6A050EDB6AD6EC0CF0C0
:10030000040EDB50025C006E050EDB50035875ECEA
:100310000BF04CEC0BF0046EFC0EDB500720056E6E
:1003200004C0E6FFE66EF6EC0CF0E9CF0AF0EACF87
:100330000BF0DB50E924086E010EDB50EA20096E59
:1003400008C0E6FFE66EB5EC39F00C6E060EE15E15
:100350000C50080EE15C02E2E16AE55220EF0BF07E
:100360006AEC0BF0080E3FEC0BF0100EF1EC0AF00B
:1003700010EC0BF0D9CFE6FFDACFE6FF64EC0BF020
:10038000030E046E25EC0DF0100EF1EC0AF025ECD6
:100390000BF003E045EC0BF0FDE13F0E00167FECA7
:1003A0000BF063EC0CF0380EEE5C000EEE58000E15
:1003B000EE58000EEE580DE2380E046E056A066A1D
:1003C000076A3CEC0DF02BEC0BF0026EEE50075878
:1003D00013D0780E086E096A0A6A0B6A3CEC0DF0BD
:1003E00084EC0DF0085C006EEE500958016EEE5082
:1003F0000A58026EEE500B58036E80EC0CF00C0E97
:10040000DBCFE6FF0D0EDBCFE6FF9D0EE66E090E9D
:10041000E66E19EC0BF06EEC0BF0080EE66EE66A79
:10042000D9CFE6FFDACFE6FF19EC0BF06EEC0BF05C
:10043000100E3FEC0BF010EC0BF0FD0EDBCFE6FFE7
:10044000FE0EDBCFE6FF64EC0BF0100EE15C02E287
:10045000E16AE55220EF0BF06AEC0BF0AFEC09F02B
:10046000EECFDFFF010EEECFDBFF020EEECFDBFFA4
:10047000030EEECFDBFF040E55EC0CF0040EEECFB6
:10048000DBFF050EEECFDBFF060EEECFDBFF070E28
:10049000EECFDBFF080E55EC0CF0080EEECFDBFFC5
:1004A000090EEECFDBFF0A0EEECFDBFF0B0EEECF19
:1004B000DBFF0C0E55EC0CF00C0EEECFDBFF0D0E3F
:1004C000EECFDBFF0E0EEECFDBFF0F0EEECFDBFF2E
:1004D000400EE66EE66AE66AE66A19EC0BF05D0E1F
:1004E000E66E090EE66E25EC08F0006E080EE15E81
:1004F0000050C9EC0BF010EC0AF0780E0026A40EA8
:1005000001226A0E0222D70EFFEC0CF003E055EC3C
:1005100009F0FDE127EC09F0190E44EC09F0FDE1CA
:1005200083EC0BF01DEC0AF0560E0026B70E0122EC
:10053000C70E0222E80E71EC0DF003E055EC09F055
:10054000FDE137EC09F0140E44EC09F0FDE19EECFE
:100550000BF02AEC0AF0DB0E0026700E0122200EB2
:100560000222240E44EC0DF003E055EC09F0FDE10D
:100570001AEC09F00F0E44EC09F0FDE1B6EC0BF0BB
:1005800037EC0AF0EE0E0026CE0E0122BD0E02223E
:10059000C10E75EC0DF003E055EC09F0FDE12AEC1D
:1005A00009F00A0E44EC09F0FDE179EC0DF044ECA1
:1005B0000AF0AF0E00260F0E01227C0E0222F50E6D
:1005C000FFEC0CF003E055EC09F0FDE127EC09F03D
:1005D000190E44EC09F0FDE183EC0BF051EC0AF04C
:1005E0002A0E0026C60E0122870E0222470E71EC4B
:1005F0000DF003E055EC09F0FDE137EC09F0140EC5
:1006000044EC09F0FDE19EEC0BF05EEC0AF0130EF9
:100610000026460E0122300E0222A80E44EC0DF0F8
:1006200003E055EC09F0FDE11AEC09F00F0E44EC83
:1006300009F0FDE1B6EC0BF06BEC0AF0002A950E28
:100640000122460E11EC0DF0160E1F0B03E055ECC7
:1006500009F0FDE12AEC09F00A0E44EC09F0FDE195
:1006600079EC0DF078EC0AF0D80E0026980E0122F5
:10067000800E0222690EFFEC0CF003E055EC09F04D
:10068000FDE127EC09F0190E44EC09F0FDE183ECE3
:100690000BF085EC0AF0AF0E0026F70E0122440E97
:1006A00002228B0E71EC0DF003E055EC09F0FDE138
:1006B00037EC09F0140E44EC09F0FDE19EEC0BF070
:1006C00092EC0AF0B10E00265B0E0122FF0E022210
:1006D00044EC0DF003E055EC09F0FDE11AEC09F0F3
:1006E0000F0E44EC09F0FDE1B6EC0BF09FEC0AF0C4
:1006F000BE0E0026D70E01225C0E0222890E75EC7A
:100700000DF003E055EC09F0FDE12AEC09F00A0ECA
:1007100044EC09F0FDE179EC0DF0ACEC0AF0220EAE
:100720000026110E0122900E02226B0EFFEC0CF03F
:1007300003E055EC09F0FDE127EC09F0190E44EC5B
:1007400009F0FDE183EC0BF0B9EC0AF0930E002602
:10075000710E0122980E7AEC0BF00C0FF4EC08F0FD
:1007600076EC09F00C0E1F0B03E055EC09F0FDE1EF
:1007700037EC09F0140E44EC09F0FDE19EEC0BF0AF
:10078000C6EC0AF08E0E0026430E0122790E0222DC
:10079000A60E44EC0DF003E055EC09F0FDE11AEC77
:1007A00009F00F0E44EC09F0FDE1B6EC0BF0D3ECD0
:1007B0000AF0210E0026080E0122B40E0222490E74
:1007C00075EC0DF003E055EC09F0FDE12AEC09F0C1
:1007D0000A0E44EC09F0FDE1EAEC0BF01DEC0AF026
:1007E000620E0026250E01221E0E0222F60E03ECDA
:1007F0000DF003E055EC09F0FDE127EC09F01B0ECC
:1008000044EC09F0FDE106EC0CF05EEC0AF0400E61
:100810000026B30E0122400E0222C00E48EC0DF05D
:1008200003E055EC09F0FDE137EC09F0170E44EC5C
:1008300009F0FDE1DDEC0BF09FEC0AF0510E002613
:100840005A0E01225E0E0222260E4CEC0DF003E041
:1008500055EC09F0FDE11AEC09F0120E44EC09F038
:10086000FDE1F2EC0BF010EC0AF0AA0E0026C70E28
:100870000122B60E0222E90E50EC0DF003E055EC19
:1008800009F0FDE12AEC09F00C0E44EC09F0FDE161
:10089000EAEC0BF051EC0AF05D0E0026100E01227E
:1008A0002F0E0222D60E03EC0DF003E055EC09F0FA
:1008B000FDE127EC09F01B0E44EC09F0FDE106EC2C
:1008C0000CF092EC0AF0530E0026140E0122440E96
:1008D0000222020E48EC0DF003E055EC09F0FDE1B8
:1008E00037EC09F0170E44EC09F0FDE1DDEC0BF0FC
:1008F000D3EC0AF0810E0026E60E0122A10E0222A0
:10090000D80E4CEC0DF003E055EC09F0FDE11AECCB
:1009100009F0120E44EC09F0FDE1F2EC0BF044ECAE
:100920000AF0C80E0026FB0E0122D30E0222E70EAB
:1009300050EC0DF003E055EC09F0FDE12AEC09F074
:100940000C0E44EC09F0FDE1EAEC0BF085EC0AF04A
:10095000E60E0026CD0E0122E10E0222210E03EC4E
:100960000DF003E055EC09F0FDE127EC09F01B0E5A
:1009700044EC09F0FDE106EC0CF0C6EC0AF0D60EF2
:100980000026070E0122370E0222C30E48EC0DF09E
:1009900003E055EC09F0FDE137EC09F0170E44ECEB
:1009A00009F0FDE1DDEC0BF037EC0AF0870E0026D4
:1009B0000D0E0122D50E0222F40E4CEC0DF003E0D8
:1009C00055EC09F0FDE11AEC09F0120E44EC09F0C7
:1009D000FDE1F2EC0BF078EC0AF0ED0E0026140EBF
:1009E00001225A0E0222450E50EC0DF003E055ECA8
:1009F00009F0FDE12AEC09F00C0E44EC09F0FDE1F0
:100A0000EAEC0BF0B9EC0AF0050E0026E90E012223
:100A1000E30E0222A90E03EC0DF003E055EC09F001
:100A2000FDE127EC09F01B0E44EC09F0FDE106ECBA
:100A30000CF02AEC0AF0F80E0026A30E0122EF0EAD
:100A40000222FC0E48EC0DF003E055EC09F0FDE14C
:100A500037EC09F0170E44EC09F0FDE1DDEC0BF08A
:100A60006BEC0AF0D90E0026020E01226F0E022254
:100A7000670E4CEC0DF003E055EC09F0FDE1DADB1C
:100A8000120E44EC09F0FDE1F2EC0BF0ACEC0AF0D4
:100A90008A0E00264C0E01222A0E02228D0E50ECE8
:100AA0000DF003E055EC09F0FDE1D4DB0C0EECDBBE
:100AB000FEE121EC0CF051EC0AF0420E0026390E5A
:100AC0000122FA0E0222FF0E07EC0DF002E0EDDB30
:100AD000FEE1BDDB1C0ED8DBFEE139EC0CF078EC5E
:100AE0000AF0810E0026F60E0122710E0222870EF8
:100AF00054EC0DF002E0D9DBFEE1B9DB150EC4DBEE
:100B0000FEE128EC0CF09FEC0AF0220E0026610EAC
:100B100001229D0E02226D0E58EC0DF002E0C5DBA5
:100B2000FEE188DB100EB0DBFEE141EC0CF0C6EC20
:100B30000AF00C0E0026380E0122E50E11EC0DF025
:100B4000170E1F0B02E0B1DBFEE184DB090E9CDB1C
:100B5000FEE121EC0CF01DEC0AF0440E0026EA0E3A
:100B60000122BE0E0222A40E07EC0DF002E09DDB76
:100B7000FEE16DDB1C0E88DBFEE139EC0CF044EC91
:100B80000AF0A90E0026CF0E0122DE0E02224B0E25
:100B900054EC0DF002E089DBFEE169DB150E74DB3D
:100BA000FEE128EC0CF06BEC0AF0600E00264B0E18
:100BB0000122BB0E0222F60E58EC0DF002E075DBAE
:100BC000FEE138DB100E60DBFEE141EC0CF092EC54
:100BD0000AF0700E0026BC0E0122BF0E0222BE0ECD
:100BE0007DEC0DF002E061DBFEE134DB090E4CDB55
:100BF000FEE121EC0CF0B9EC0AF0C60E00267E0EE8
:100C000001229B0E0222280E07EC0DF002E04DDBC4
:100C1000FEE11DDB1C0E38DBFEE139EC0CF010ECC4
:100C20000AF0FA0E0026270E0122A10E0222EA0E79
:100C300054EC0DF002E039DBFEE119DB150E24DB8C
:100C4000FEE128EC0CF037EC0AF0850E0026300EA1
:100C50000122EF0E0222D40E58EC0DF002E025DB4B
:100C6000FEE1E8DA100E10DBFEE141EC0CF05EEC88
:100C70000AF0050E00261D0E0122880E0222040E27
:100C80007DEC0DF002E011DBFEE1E4DA090EFCDAA6
:100C9000FEE121EC0CF085EC0AF0390E0026D00EB6
:100CA0000122D40E0222D90E07EC0DF002E0FDDA8B
:100CB000FEE1CDDA1C0EE8DAFEE139EC0CF0ACEC2A
:100CC0000AF0E50E0026990E0122DB0E0222E60E46
:100CD00054EC0DF002E0E9DAFEE1C9DA150ED4DADF
:100CE000FEE128EC0CF0D3EC0AF0F80E00267C0EA6
:100CF0000122A20E02221F0E58EC0DF002E0D5DAFE
:100D0000FEE198DA100EC0DAFEE141EC0CF0A2DB55
:100D1000650E0026560E0122AC0E0222C40E7DEC9A
:100D20000DF002E0C2DAFEE195DA090EADDAFEE17D
:100D30000FEC0CF075DB440E0026220E0122290E6A
:100D40000222F40E0CEC0DF002E0AFDAFEE17FDAE5
:100D50001A0E9ADAFEE1FAEC0BF0BDDB970E0026D4
:100D6000FF0E01222A0E0222430E5CEC0DF002E07F
:100D70009CDAFEE17CDA160E87DAFEE12FEC0CF04D
:100D8000C6EC0AF0A70E0026230E0122940E0222C2
:100D9000AB0E60EC0DF002E088DAFEE14BDA110EEA
:100DA00073DAFEE118EC0CF07CDB390E0026A00EA5
:100DB0000122930E0222FC0E64EC0DF002E075DAC3
:100DC000FEE148DA0B0E60DAFEE10FEC0CF0C4DB5A
:100DD000C30E0026590E01225B0E0222650E0CEC9A
:100DE0000DF002E062DAFEE132DA1A0E4DDAFEE1CF
:100DF000FAEC0BF03CDB920E0026CC0E01220C0E1E
:100E000002228F0E5CEC0DF002E04FDAFEE12FDAE9
:100E1000160E3ADAFEE12FEC0CF084DB7D0E002694
:100E2000F40E0122EF0E0222FF0E60EC0DF002E044
:100E30003CDAFEE1FFD9110E27DAFEE118EC0CF0E6
:100E4000FCDAD10E00265D0E0122840E0222850EF0
:100E500064EC0DF002E029DAFEE1FCD90B0E14DAA5
:100E6000FEE10FEC0CF044DB4F0E00267E0E01225B
:100E7000A80E02226F0E0CEC0DF002E016DAFEE175
:100E8000E6D91A0E01DAFEE1FAEC0BF08CDBE00E8B
:100E90000026E60E01222C0E0222FE0E5CEC0DF066
:100EA00002E003DAFEE1E3D9160EEED9FEE12FEC03
:100EB0000CF004DB140E0026430E0122010E022268
:100EC000A30E60EC0DF002E0F0D9FEE1B3D9110EF3
:100ED000DBD9FEE118EC0CF04CDBA10E0026110E64
:100EE0000122080E02224E0E64EC0DF002E0DDD964
:100EF000FEE1B0D90B0EC8D9FEE10FEC0CF0C4DA5C
:100F0000820E00267E0E0122530E0222F70E0CECFA
:100F10000DF002E0CAD9FEE19AD91A0EB5D9FEE168
:100F2000FAEC0BF00CDB350E0026F20E01223A0E25
:100F30000222BD0E5CEC0DF002E0B7D9FEE197D9BC
:100F4000160EA2D9FEE12FEC0CF084DABB0E0026BF
:100F5000D20E0122D70E02222A0E60EC0DF002E022
:100F6000A4D9FEE167D9110E8FD9FEE118EC0CF07F
:100F7000CCDA910E0026D30E0122860E0222EB0E51
:100F800064EC0DF002E091D9FEE164D90B0E7CD93E
:100F9000FEE10BD9E4D9C0EC0CF0040E55EC0CF0DA
:100FA000A7EC0CF0080E55EC0CF09AEC0CF00C0EC3
:100FB00055EC0CF08DEC0CF0100EE15C02E2E16AF5
:100FC000E5523ED312DBFCDA3AE2DFCF06F0010E47
:100FD000DBCF07F0D89006360736D89006360736AE
:100FE000FB0EDB50062413EC0DF00720EA6EEECF6B
:100FF00002F00250E66EDDEC0CF0B8D9080E44D9D0
:10100000FEE10450E66E010E49EC0CF0AFD9100E73
:101010003BD9FEE10450E66E020E49EC0CF0A6D975
:10102000180E32D9FEE10450E66E030E49EC0CF0C6
:1010300077EC0CF0E552E750EF6EE4DAC4D7080E17
:10104000E15C02E2E16AE552FBD2CFDAB9DA01E310
:10105000A2D022DB13EC0DF00720EA6EEFCF02F0F6
:10106000036A046A056A010E0C6E0D6A0E6A0F6A45
:1010700033EC0DF0EE500C26EE500D22EE500E2209
:10108000EE500F22FB0EDB500C2413EC0DF00D2064
:10109000EA6EEFCF08F0096A0A6A0B6A080E1F0BA6
:1010A00002E004DBFEE108500212095003120A506C
:1010B00004120B500512020E146E156A166A176A96
:1010C00033EC0DF0EE501426EE501522EE501622A1
:1010D000EE501722FB0EDB50142413EC0DF01520FC
:1010E000EA6EEFCF10F0116A126A136A100E1F0B2E
:1010F00007E0D8901036113612361336E806F9E1BB
:101100001050021211500312125004121350051203
:10111000030E1C6E1D6A1E6A1F6A33EC0DF0EE5042
:101120001C26EE501D22EE501E22EE501F22FB0EFA
:10113000DB501C2413EC0DF01D20EA6EEFCF18F0ED
:10114000196A1A6A1B6A180E1F0B07E0D890183626
:1011500019361A361B36E806F9E1185002121950F2
:1011600003121A5004121B500512DFCF00F0010EBB
:10117000DBCF01F0D89000360136D890003601362A
:10118000B6DB02C0EEFF03C0EEFF04C0EEFF05C0F9
:10119000EEFF38DA5BD7080EE15C02E2E16AE55265
:1011A0004FD288DB90DB8DEF0CF084DB040E00C0A7
:1011B000DBFF050E01C0DBFF060E02C0DBFF070EE2
:1011C00003C0DBFF33EC0DF09AEF0CF073DB98DB20
:1011D00068EC0DF0DACFEAFFC0EF0CF06BDBC4DB9C
:1011E00037EC0DF0A7EF0CF0E96EDACFEAFFEDEF88
:1011F0000CF0DACFEAFF0C50EE14086E0D50EE142E
:10120000096E0E50EE140A6E0F50EE140B6EC4D31E
:1012100003220050DE260150DE220250DE2203505F
:10122000DD22DD52DD5237EC0DF02CEC0DF0EFCF6E
:1012300003F01200080EDBCF04F0090EDBCF05F03F
:101240000A0EDBCF06F00B0EDBCF07F0120037ECF7
:101250000DF0BAD3040EDBCF04F0050EDBCF05F0A2
:10126000060EDBCF06F0070EDBCF07F012000C0EE8
:10127000DBCF04F00D0EDBCF05F00E0EDBCF06F05A
:101280000F0EDBCF07F01200D8900732063205327E
:101290000432E806120084EC0DF00816EE50091630
:1012A000EE500A16EE500B1677D3D8900036013662
:1012B00002360336E806120084EC0DF00416EE50F8
:1012C0000516EE500616EE5007161200DACFEAFFAA
:1012D0000850EE18046E0950EE18056E0A50EE180C
:1012E000066E0B50EE18076E045012000C0EDBCF8A
:1012F00000F00D0EDBCF01F00E0EDBCF02F00F0E73
:10130000DBCF03F01200080EDBCF00F0090EDBCFBD
:1013100001F00A0EDBCF02F00B0EDBCF03F0120060
:101320004CDB17EF0DF0F0DB041AEE50051AEE500F
:10133000061AEE50071A04501200E6DB081AEE50A7
:10134000091AEE500A1AEE500B1A1200DDDB0412D5
:10135000EE500512EE500612EE5007121200FD0E6E
:10136000DBCFE9FFFE0EDBCFEAFF1200C0DAE55269
:10137000E750EF6EDFCF08F0010EDBCF09F0D89019
:1013800008360936D89008360936FB0EDB5008249B
:101390004ADB0920EA6E18D30C0EDBCF08F00D0EE5
:1013A000DBCF09F00E0EDBCF0AF00F0EDBCF0BF018
:1013B0001200080EDBCF08F0090EDBCF09F00A0E91
:1013C000DBCF0AF00B0EDBCF0BF01200040EDBCFED
:1013D00008F0050EDBCF09F0060EDBCF0AF0070E92
:1013E000DBCF0BF0120043DBEECF08F0EECF09F0BD
:1013F000EECF0AF0EFCF0BF01200DBCF0FF00C1E98
:101400000D1E0E1E0F1E1200081E091E0A1E0B1EA8
:10141000D9501200041E051E061E071ED9501200C8
:1014200009015D25006E05505E21016E06505F21A9
:10143000026E07506021036E120009016125006EE3
:1014400005506221016E06506321026E075064212F
:10145000036E120009016525006E05506621016EBC
:1014600006506721026E07506821036E12000901C1
:101470006925006E05506A21016E06506B21026ECF
:1014800007506C21036E120009016D25006E055096
:101490006E21016E06506F21026E07507021036E9F
:1014A000120009017125006E05507221016E06506F
:1014B0007321026E07507421036E12000901752515
:1014C000006E05507621016E06507721026E07509E
:1014D0007821036E120009017925006E05507A21EA
:1014E000016E06507B21026E07507C21036E1200B4
:1014F00009017D25006E05507E21016E06507F2179
:10150000026E07508021036E120009018125006ED2
:1015100005508221016E06508321026E07508421FE
:10152000036E120009018525006E05508621016EAB
:1015300006508721026E07508821036E12000901B0
:101540008925006E05508A21016E06508B21026E9E
:1015500007508C21036E120009018D25006E055085
:101560008E21016E06508F21026E07509021036E6E
:10157000120009019125006E05509221016E06505E
:101580009321026E07509421036E120009019525E4
:10159000006E05509621016E06509721026E07508D
:1015A0009821036E120009019925006E05509A21B9
:1015B000016E06509B21026E07509C21036E1200A3
:1015C000F70EDBCF00F0F80EDBCF01F0EFD94BDAEE
:1015D0000050EE5C0150EE580250EE580350EE58A9
:1015E0001200E926000EEA22120004DA080EE126B3
:1015F00025DA040EDB6A050EDB6A060EDB6A070ECF
:10160000DB6A120034DAEE2A000EEE22EE22EE221F
:101610002ADA040EEE26000EEE22EE22EE22120050
:10162000E9CF00F0EACF01F0E9CFE6FFEACFE6FF2D
:101630001200FB0EDBCFE6FFFC0EDBCFE6FF120055
:10164000E16EE552E7CFD9FF120004501F0B04DA18
:10165000EECF03F0120058DA045C006EEE5005582D
:10166000016EEE5006581200E9CFE6FFEACFE6FF22
:101670002CEC02F0E552E552E552E5521200E66E1E
:10168000E66AE66AE66A25EF0DF0D8900332023288
:1016900001320032E8061200040EDBCF06F0050E20
:1016A000DBCF07F0FB0EDB5006241200D890083683
:1016B00009360A360B36E8061200F90EDBCF00F0C9
:1016C000FA0EDBCF01F012007DDC026E080EE15E47
:1016D000025012008FD9100EE126120083EC00F0A8
:1016E000006E060EE15E00501200016E00C0E6FFC3
:1016F000E66E12000222FD0E0322D9501200016A8A
:10170000026A036A12006ADDA5DDD9CFE9FFD4DDE4
:10171000AED9EECF0CF0EECF0DF0EECF0EF0EFCF56
:101720000FF00C1E0D1E0E1E0F1EA6D9F9EF08F0AD
:101730000322D950080F58DD83EF09F047DD87DD1C
:10174000C7D9BADD0C0EDBCF0CF00D0EDBCF0DF0E0
:101750000E0EDBCF0EF00F0E50DEDAD9F9EF08F0E7
:101760000322D9500C0F40DD76EF09F01ADD7FDD42
:1017700083D9A2DD080EDBCF0CF0090EDBCF0DF014
:101780000A0EDBCF0EF00B0E38DED9CFE9FFF9EFF2
:1017900008F050DDBDD990DD040EDBCF0CF0050E56
:1017A000DBCF0DF0060EDBCF0EF0070E26DE90D954
:1017B000F9EF08F00322D9508FD108DD4BDD88D92D
:1017C0007BDD04DE081E091E0A1E0B1ED9CFE9FFB1
:1017D0004BEF09F0EADC4BDD9BD96EDDDDDD14DE7D
:1017E000080F8FD1DEDC33DD47D966DDFCDD0CDE92
:1017F0000C0F87D1F3DC1EDD041E051E061E071E1E
:10180000D9CFE9FFA3DD84D993EF09F0E7DC12DD3E
:10181000D9CFE9FF51DDCDDDF7DD040F72D1C5DC95
:1018200026DDF8DD040FE96E91DD26D993EF09F08E
:10183000B8DC0DDDEFDD080FE96E88DD49D993EFE7
:1018400009F0B3DCB6DD64D978DD42D966EF09F082
:10185000BDDCC9DD3DD971DD5BD966EF09F0B6DCD1
:10186000F9DCD8DD0C0FE96E71DDD9CFE9FF93EF1C
:1018700009F0B4DCABDDD9CFE9FF5FDDFDD866EF61
:1018800009F08FDC89DDF8D858DDD9CFE9FF66EFA4
:1018900009F0006E34DFE7D8EE500026EE5001224A
:1018A000EE500222EE5003221200E76E58DDE750A0
:1018B000F1EF0AF004500012055001120650021216
:1018C000075003121200080E00C0DBFF090E01C012
:1018D000DBFF0A0E02C0DBFF0B0E03C0DBFFCCD820
:1018E000DACFEAFF12003BDD100EF1EF0AF0FD0E39
:1018F000DB500024E96EFE0EDB500120EA6E120080
:101900000C0E00C0DBFF0D0E01C0DBFF0E0E02C08F
:10191000DBFF0F0E03C0DBFF12000C0EDB50EE26C8
:101920000D0EDB50EE220E0EDB50EE220F0EDB50C2
:10193000EE221200080EDB50EE26090EDB50EE22DE
:101940000A0EDB50EE220B0EDB50EE221200040ECC
:10195000DB50EE26050EDB50EE22060EDB50EE22AB
:10196000070EDB50EE22120000C0DFFF010E01C0A7
:10197000DBFF020E02C0DBFF030E03C0DBFF120021
:10198000DF50EE26010EDB50EE22020EDB50EE227F
:10199000030EDB50EE22120008500412095005120B
:1019A0000A5006120B50071204501200F90EDBCF3A
:1019B00002F0FA0EDBCF03F01200040EDBCF00F0D2
:1019C000050EDBCF01F01200EECF04F0EECF05F0F4
:1019D000EECF06F0EFCF07F012000050EE260150D8
:1019E000EE220250EE220350EE221200B8DC180E56
:1019F000F1EF0AF0D9CFE6FFE1CFD9FF120008DC02
:101A0000070E1F0B120004DC050E1F0B120008EC62
:101A100009F0040E1F0B120008EC09F0060E1F0B54
:101A2000120068DE59D0E96EFC0EDB501200060E83
:101A3000DBCF02F0070EDBCF03F01200DE6ADE6AB6
:101A4000DE6ADD6ADD52DD521200FB0EDBCFE9FFFC
:101A5000FC0EDBCFEAFF1200EECF00F0EECF01F07C
:101A6000EECF02F0120054D8DACFEAFF1200D9CF3D
:101A7000E9FFDACFEAFF1200D950080FE96E120031
:101A800032DF040EF1EF0AF053DE110E1F0B1200CD
:101A900067DE090E1F0B12004BDE0E0E1F0B12002D
:101AA00089DE140E1F0B12005BDE0B0E1F0B1200E3
:101AB0003FDE100E1F0B120053DE0A0E1F0B12002A
:101AC00037DE0F0E1F0B120075DE150E1F0B1200F6
:101AD000D9500C0FE96E1200040FF4EC08F090EFEF
:101AE00009F03EDE0C0E1F0B120064DE160E1F0BFB
:101AF0001200D5EC08F0C9EF0BF05CDE170E1F0BDF
:101B00001200E96E4BEF09F0DACFEAFFEE50120057
:081B1000D950040FE96E120028
:081B18000601F96BFA6B1200E3
:101B20000601C86B12000601010EC96F050E0BEC11
:101B300017F00501440EFE6F610E54EC17F00A0E0B
:101B40000BEF17F00501420EFE6F610E54EF17F018
:101B50006FEC16F0030EE1260601F80548E1450E8C
:101B60000601055D44E0410E055D41E0610E055D45
:101B70003EE0670E055D3BE0500E055D38E0020E6D
:101B800005C6DBFF060EE66E060EE66E000EE66E7E
:101B9000050E1FEC17F09AEC16F0EAEC16F002E6D0
:101BA00060EC17F005E203EC18F0F7E3DB2AF5D759
:101BB00087EC18F094EC3AF01DEC18F0000EE66E8D
:101BC000050E30EC16F03A0E006E610EDCEC17F0EC
:101BD000020EDBCF07F6080EE66E060EE66EC4ECCC
:101BE00016F087EC18F042EC32F024EC17F07FECA2
:101BF00018F094EC3AF01DEC18F0E4EC16F0C4EC9C
:101C000016F07FEC18F078EC17F0370EFE6F610ECF
:101C100054EC17F0030EE15C02E2E16AE55248EF92
:101C200016F06FEC16F0050EE126D650016E006A34
:101C3000030E00C0DBFF040E01C0DBFFD75029EC10
:101C400017F0DF6A080EDF5C0BE2DF50EA6ADD0F97
:101C5000E96E080EEA22EF5029EC17F0DF2AF2D7DE
:101C6000030EDBCFE6FF040EDBCFE6FF44EC44F0CF
:101C7000E552E552DF6A160EDF5C0DE274EC16F0F9
:101C8000DF50EA6ACA0FE96E060EEA22E552E75013
:101C9000EF6EDF2AF0D70601E06B090E2DEC18F08D
:101CA000D80EE66E040EE66E46EC17F094EC3AF0B1
:101CB0004AEC16F046EC17F0160EE66EE66A65EC96
:101CC00017F052EC42F0026E0A0EE15E025005017E
:101CD0002F0EFE6F610E54EC17F065EC17F019EC47
:101CE00017F02D0EFE6F610E54EC17F0F5EC16F0A8
:101CF00078EC17F02D0EFE6F610E54EC17F0080E05
:101D00002DEC18F046EC17F019EC17F0370EFE6FBB
:101D1000610E54EC17F0050EE15C02E2E16AE55257
:101D200048EF16F029EC18F0260E006E610EDCEC80
:101D300017F045EC18F009010551E66EE66A03C993
:101D4000E6FF04C9E6FFC4EC16F06AEC17F0190EC2
:101D5000006E610E10EC16F00D0EE15E035000EC0B
:101D600016F0090109510F0A18E0020A12E0090AE7
:101D70000CE0060A06E0030A14E10F0E006E610E85
:101D800013D0070E006E610E0FD0010E006E610EB3
:101D90000BD0F80E006E600E07D0EF0E006E600ED6
:101DA00003D0E60E006E600E84EC18F009010B51B2
:101DB000040A12E0070A0CE0020A06E0010A10E138
:101DC000DC0E006E600E0FD0D30E006E600E0BD0D6
:101DD000CC0E006E600E07D0BF0E006E600E03D0FA
:101DE000BD0E006E600E84EC18F08FEC16F04D08FE
:101DF0000AE114C9E6FF15C9E6FFB90E006E600ED0
:101E000010EC18F00AD014C900F015C901F0040E46
:101E1000ABEC17F0FDE1AAEC18F000EC16F08FEC3B
:101E200016F04D080AE116C9E6FF17C9E6FFB90E1C
:101E3000006E600E10EC18F00AD016C900F017C939
:101E400001F0040EABEC17F0FDE1AAEC18F000EC89
:101E500016F058C900F0016A00BE01680BEC18F0DA
:101E600051C9E6FF52C9E6FF50C902F0036A02BE3B
:101E7000036802C0E6FF03C0E6FF09010B51E66EEE
:101E8000E66A09010951E66EE66A09010A51E66E41
:101E9000E66A09010D51E66EE66A09010C51E66E2B
:101EA000E66A07C9E6FF08C9E6FF09010651E66EC2
:101EB000E66A9B0E046E600E056E066A04C0E6FFBD
:101EC000E66E06C0E6FFFBEC17F0076E190EE15E4A
:101ED00007508CEC18F0020EE15C02E2E16AE55278
:101EE00048EF16F0940E006E600EDCEC17F0BEECBE
:101EF00017F056C900F0016A00BE0168FDEC16F04B
:101F0000870E026E600E06EC16F00D0EE15E0550B7
:101F10008CEF18F06FEC16F0090EE126090136512E
:101F200007E1375105E1385103E1395101E18AD028
:101F3000800E006E600EDCEC17F0DF6A040EDF5CD2
:101F400073E28FEC17F0EFCF00F0000EE76E001891
:101F5000E8AE02D0003403D0E750D88000545DE2F0
:101F6000DF50EA6A3A0FE96E090EEA22EFCF04F079
:101F700004C029F0A2EC34F027C000F028C001F022
:101F800029C002F02AC003F0560E2C6E0E0E2D6EE4
:101F90008D0E2E6E3E0E2F6EE3EC34F035EC36F0E7
:101FA000010E26C0DBFF020E27C0DBFF030E28C098
:101FB000DBFF040E29C0DBFFD1EC16F0050E26C0B6
:101FC000DBFF060E27C0DBFFD1EC16F0070E22C0A8
:101FD000DBFF080E23C0DBFF8FEC17F0EF50D80FAC
:101FE000006E016A00BE01680BEC18F0070EDBCF33
:101FF000E6FF080EDBCFE6FF050EDBCFE6FF060EA1
:10200000DBCFE6FF760E026E600E06EC16F00B0ECE
:10201000E15E055000EC16F005D0710E006E600E0A
:1020200084EC18F0DF2A8AD757C900F0016A00BE95
:1020300001680BEC18F06E0E026E600E15EC18F0D5
:102040008CEC18F0090EE15C02E2E16AE55248EF1F
:1020500016F0670E006E600EDCEC17F0C70EE66E31
:10206000080EE66E0801DB51E66EE66A09015C5176
:10207000E66EE66A210EE66E090EE66E0901025171
:10208000E66EE66A0151E66EE66A0051E66EE66AC1
:10209000520E006E600E10EC16F0130EE15E03504F
:1020A0008CEF18F06FEC16F0040EE12609011C51BC
:1020B0001D111E111F1107E1DE6ADE6ADE6ADD6A8C
:1020C000DD52DD521CD01C0EE96E090EEA6EEE5098
:1020D0000901185D006EEE501959016EEE501A5943
:1020E000026EEE501B59036E00C0DFFF010E01C0EF
:1020F000DBFF020E02C0DBFF030E03C0DBFF4B0E53
:10210000006E600EDCEC17F054C900F0016A00BEEE
:1021100001680BEC18F055C902F0036A02BE0368AF
:1021200002C0E6FF03C0E6FF09011051E66EE66A51
:1021300020C904F0056A04BE056804C0E6FF05C0B6
:10214000E6FF6FEC17F0EECFE6FFEECFE6FFEECF47
:10215000E6FFEFCFE6FF09011251E66EE66A40C9DD
:10216000E6FF41C9E6FF42C9E6FF43C9E6FF3EC9B3
:10217000E6FF3FC9E6FF35C906F0076A06BE0768F5
:1021800006C0E6FF07C0E6FF09013451E66EE66AC5
:1021900033C908F0096A08BE096808C0E6FF09C02B
:1021A000E6FF09011151E66EE66A09010F51E66E7C
:1021B000E66A09010E51E66EE66A1F0E0A6E600EAF
:1021C0000B6E0C6A0AC0E6FFE66E0CC0E6FFFBEC85
:1021D00017F00D6E250EE15E0D508CEC18F0040E1C
:1021E000E15C02E2E16AE55248EF16F06FEC16F0AE
:1021F000180E006E600EDCEC17F056C900F0016A94
:1022000000BE0168FDEC16F009011251E66EE66AA7
:102210006AEC17F029EC16F0020E026E600E06EC66
:1022200016F0130EE15E055000EC16F0BEEC17F050
:102230008FDC76EF18F06FEC16F0060E96EC17F0C8
:102240008FEC16F009E08FEC16F0200805E0DF2A8D
:10225000010EF6E3DB2AF4D78FEC16F0200801E03C
:10226000C7D09DEC17F001E3DB2AEF6A29EC16F0EA
:1022700065EC17F07DEC17F001E1BAD0090EE66EBF
:10228000A5EC16F0D80EE66E040EECEC17F029EC77
:1022900016F0AFEC16F029EC16F04DEC17F07FECD1
:1022A00018F0F5EC16F042EC32F024EC17F07FEC6D
:1022B00018F0C4EC16F07DEC17F001E099D029EC91
:1022C00016F0000EE66E060E1FEC17F065EC17F028
:1022D000D7EC17F0D80EE66E040EECEC17F07FEC9E
:1022E00018F0AFEC16F07FEC18F04DEC17F0F5ECB1
:1022F00016F04CEC18F035EC17F010EC17F002E685
:1023000060EC17F00AE2A4EC18F0E7EC16F0040E0B
:10231000DB2A050EF2E3DB2AF0D7F5EC16F054ECDD
:1023200018F035EC17F010EC17F002E660EC17F03F
:102330000AE2A4EC18F0E4EC16F0040EDB2A050E19
:10234000F2E3DB2AF0D70601010EC86F0A0EE66E33
:10235000A5EC16F003EC16F0500848E10601F85120
:1023600023E1040EDB6A050EDB6A10EC17F004E6CD
:10237000160E005C000E015815E274EC16F0040E07
:10238000DBCFE9FF050EDBCFEAFFE10EE926060E03
:10239000EA22E552E750EF6E040EDB2A050EE5E374
:1023A000DB2AE3D70601F76BF86BFA0E006E5F0EBF
:1023B000DCEC17F0B0EC17F0D7EC17F093EC0DF065
:1023C00074EC17F00601010EF86FE66EA5EC16F03E
:1023D000E80EE66E040EECEC17F0B0EC17F0AFEC84
:1023E00016F0B0EC17F04DEC17F002D00601F86BC8
:1023F000060EE15C02E2E16AE55248EF16F029ECD4
:1024000018F00601C85114E1070EE66EE66AF20EF6
:10241000006E5F0EDFEC17F029EC16F082EC17F07F
:1024200001E0A6D0070E62EC16F005DFE5521CD0E5
:1024300094EC18F07FEC18F029EC16F0FEEC32F07A
:10244000E552E5521DEC18F0E7EC16F0050EE66ECD
:10245000E66AEC0E006E5F0ED0DB82EC17F006E051
:10246000400EE66E59EC1AF0E55282D0D950FD0FBD
:10247000E96EDACFEAFF050EEE6E060EED6EEEECBB
:1024800016F0EF5045083DE15CEC18F04D0839E1DD
:10249000D950FD0FE96EFF0EDA20EA6E020EEE262D
:1024A000000EED2294EC18F0010EE66E050EE66EBD
:1024B000010E62EC16F0FEEC32F08FEC18F0CCEC72
:1024C00016F09AEC16F0EAEC16F002E660EC17F063
:1024D00005E203EC18F0F7E3DB2AF5D7C4EC16F0BD
:1024E000010EE66E050EBCDBEEEC16F0EFCF00F54C
:1024F000D950FD0FE96EDACFEAFF000EEE6E050E41
:10250000ED6EEEEC16F0EF50430A29E0190A0FE0E9
:102510001B0A2EE1E50E006E5F0EDCEC17F00601E3
:10252000C95126E193EC0DF0A8EC0DF012D05CEC53
:1025300018F0300811E00901010E5B6F0601C95166
:1025400017E193EC0DF092EC0EF0CCDCE3DC81DDD6
:10255000A9DDA2EC0DF00CD009015B6B09D0010ED6
:10256000B1DB0CD8E552E5520601C95101E130D882
:10257000020EE15C02E2E16AE5528AD3B0DB040EAE
:1025800096EC17F0CCDB08E0CADB2C0805E0DF2A6C
:10259000010EF8E3DB2AF6D7C2DB2C0805E19DEC3F
:1025A00017F001E3DB2AEF6A54DB39EC18F0F3CFC4
:1025B000F9F6F4CFFAF6C4EC16F0600EE66E000EF3
:1025C0001FEC17F0040EE15C02E2E16AE55260D311
:1025D00086DB040EE126020E0BEC17F0280E060136
:1025E000FAAF02D0D89003D0F95D000EFA5907E394
:1025F000FA3507E2F9513108000EFA5502E293EC80
:102600000DF0310E0601F91901E1FA5101E124D270
:10261000290EF91901E1FA5101E113D2280EF91935
:1026200001E1FA5101E1ECD1180EF91901E1FA5179
:1026300001E1D8D1170EF91901E1FA5101E1BCD13C
:10264000160EF91901E1FA5101E1B0D1150EF9198F
:1026500001E1FA5101E1A4D1140EF91901E1FA5195
:1026600001E198D1130EF91901E1FA5101E18CD180
:10267000120EF91901E1FA5101E180D1110EF91997
:1026800001E1FA5101E159D1100EF91901E1FA51B4
:1026900001E136D10F0EF91901E1FA5101E12AD118
:1026A0000C0EF91901E1FA5101E110D10B0EF919E3
:1026B00001E1FA5101E1F1D00A0EF91901E1FA51F3
:1026C00001E1E3D0050EF91901E1FA5101E1D5D09C
:1026D000040EF91901E1FA5101E198D0030EF9193C
:1026E00001E1FA5101E16FD0020EF91901E1FA514D
:1026F00021E0010EF91901E0BED1FA5101E0BBD190
:10270000DE6ADD6A67DB04E6100E005C000E01582D
:1027100001E3B9D1CCDBEF50E66EE66A100EE66E4F
:10272000E66A32DBD20E006E5F0E67DAA4DBEAE304
:10273000DB2AE8D7BDDA67DA08E01AEC18F005E022
:10274000BAEC17F0F8E3DB2AF6D71AEC18F001E040
:1027500010D112DB01E3DB2A62EC18F001E088D033
:10276000A4EC17F004E6100E025C000E035801E31F
:102770007FD061DA39EC18F0F350E66E98DBE55261
:10278000E750EF6E27DB04E6080E005C000E0158F0
:102790000FE351DA7AEC18F0080E005E000E015AD1
:1027A000180E0024E66EE8EC3FF0E552E552E552E3
:1027B00096DB0F0EEE1801E021D1ED5001E01ED1A5
:1027C000A7EC3BF01BD1DE6ADD6A04DB04E6200ED9
:1027D000005C000E015801E356D1DFCFE6FFB5DA09
:1027E0007EDB090EEE1805E1ED5003E16FEC18F009
:1027F000EF6A21DA200EE66EE66AC6DABF0E006ED8
:102800005F0EFBD938DBE1E3DB2ADFD751DAFBD9F6
:1028100007E01AEC18F004E0ADDBF9E3DB2AF7D7A8
:102820001AEC18F001E0A5D0A7DA01E3DB2A62EC8C
:1028300018F01EE189DB04E6180E025C000E035856
:1028400017E2F9D9DFCFE6FFE8EC3FF0E552E552B9
:10285000E552D4DBD2D922EC18F041DB020EEE189F
:1028600001E00FD1ED5001E00CD1A7EC3BF009D114
:102870005CDA0B0E006E890E02D1C0DBBED989DA9C
:10288000040EE66E59EC1AF0F4D00801DB5101E1B8
:10289000ACD0F4DBC3EC3CF0B0D00801DB5101E17B
:1028A000A4D0040E09010E150CE0070E09010A5D03
:1028B00008E0010EE66EC5EC3CF0E5520701F06B56
:1028C0009DD033DA2D0E006E890ED9D00801DB5170
:1028D00001E18BD009010EA908D0E66AC5EC3CF0F5
:1028E000E55207011E0EF06F89D01FDA5B0E006EF5
:1028F000890EC5D00801DB5101E177D068DB17D024
:102900000801DB5172E0D4D97ED906E093DB04E004
:1029100031DBFAE3DB2AF8D78DDB2BE12DDA01E39B
:10292000DB2AEF6AABDBC3EC3CF0E55284D9A1DBD8
:10293000F350E66EC4EC3CF060D00801DB5155E08A
:10294000B7D961D906E076DB04E014DBFAE3DB2AD1
:10295000F8D770DB0EE110DA01E3DB2AEF6A6BD9FE
:10296000CFEC43F097D98ADBC7EC3CF0E552E55257
:1029700044D0DBD9CF0E006E880E81D00801DB5128
:1029800034E0C1EC3CF003D00801DB512EE0C2EC96
:102990003CF034D00801DB5112E019DB020E16D0F6
:1029A0000801DB510CE013DBE66A11D00801DB51B2
:1029B00006E00DDB030E0AD00801DB5105E1B5D9B5
:1029C000E90E006E880E09D002DB010EE66EC6EC41
:1029D0003CF0E552E552E55211DB47DB1CDA52ECE4
:1029E00010F051D00801DB5105E19FD9E90E006ECE
:1029F000880E45D043DBC8EC3CF0E552FFDA3FD00F
:102A000057D901D906E016DB04E0B4DAFAE3DB2A91
:102A1000F8D710DB0FE1B0D901E3DB2AEF6AD7DA90
:102A20003EEC21F0E552E55206D903DA420EFE6F84
:102A3000610E17D093EC0DF078D9CF0E006E880E92
:102A400014D00501B30EFE6F5F0E2EDAC0DAF1D995
:102A5000AD0EFE6F5F0E05D0BADAEBD9AB0EFE6F8E
:102A60005F0E22DA050E0EDBC9DAFFDAE66E5FECE6
:102A70003EF0E55208D059D9A00E006E5F0EBDD8C9
:102A8000E1DAA8EC0DF0A2EC0DF00601F96BFA6B9F
:102A90000001606B040EE15C02E2E16AE552F8D0ED
:102AA0001ED90601C85121E0C95100081EE3020EDB
:102AB00057DB8D0E006E5F0E27DBCBD878DA840EE5
:102AC000006E5F0E21DBAA0EE76EFB0EDBCFE9FF87
:102AD000FC0EDBCFEAFF49DAEF6AFB0EDBCFE6FF45
:102AE000FC0EDBCFE6FF63DAFFD900D3B2DA38DBC6
:102AF00009010B51040A12E0070A0CE0020A06E081
:102B0000010A10E1780E006E5F0E0BD06D0E006EA4
:102B10005F0E07D0640E006E5F0E03D0550E006E80
:102B20005F0EF2DA090109510F0A18E0020A12E0F9
:102B3000090A0CE0060A06E0030A14E14C0E006ED6
:102B40005F0E13D0360E006E5F0E0FD0280E006E93
:102B50005F0E0BD01E0E006E5F0E07D00C0E006EC7
:102B60005F0E03D0FB0E006E5E0ECEDAEC0E006E32
:102B70005E0ECADA8ADAD3D84D0809E114C9E6FF35
:102B800015C9E6FFE60E006E5E0E4ADA0CD014C9D7
:102B900000F015C901F0040EDED9FEE163D8E00EA5
:102BA000026E5E0E42DA2CD8D90E006E5E0EACDAE2
:102BB00091D9D40E006E5E0E33DA22D895D9020E6A
:102BC000E15C02E2E16AE55263D043DA5BDAA90E26
:102BD000006E5E0EF1D988D9020EE15C02E2E16A74
:102BE000E55256D036DA76D9700E006E5E0E3DDABA
:102BF000E15C02E2E16AE5524BD0E1D97FEF18F0E7
:102C000086DAD7EF17F06BDAEF501200036E046A22
:102C100002C0E6FFE66E04C0E6FFEDD9056E1200C5
:102C2000CED9E9D9036E12001EEC3AF0036E050E00
:102C3000E15E03501200020EDBCFE6FF030EDBCF96
:102C4000E6FF12007BEC3AF0036E050EE15E0350E6
:102C50001200FD0EDBCFE6FFFE0EDBCFE6FF12001B
:102C60006ADAC1D1050E0026000E01220A0E2D6E71
:102C70002E6A00C028F001C029F0D5EC46F028C02B
:102C800000F029C001F028C0E6FF29C0E6FF1200CD
:102C9000E16E2CD2E552E552F3CF00F0F4CF01F013
:102CA000F3CFE6FFF4CFE6FF120091D939EF18F029
:102CB000D950020FE96EDACFEAFF600EEE6E000E19
:102CC000ED6E1200E76EFD0EDBCF00F0FE0EDBCFE7
:102CD00001F0E7500026000E01220BEF18F0D9CFCB
:102CE000E6FFE1CFD9FF12004BEC44F0F3CFF6FF43
:102CF000F4CFF7FF400E2D6E2E6AF6CF28F0F7CFF7
:102D000029F0BDEC35F024C0F6FF25C0F7FF7A0EA0
:102D1000F6268B0EF7220800F550E66E1200DECF85
:102D2000E9FFDDCFEAFFEF501200F9C6E6FFFAC671
:102D3000E6FF1200100EE66EE66AE80EE66E040E7E
:102D4000FAD9C5D9DE6ADD6A1200A3EC3FF0E5527C
:102D5000020EF3CFDBFF030EF4CFDBFF120094EC87
:102D60003AF0E552E552F3CF02F0F4CF03F0F3CF9F
:102D7000E6FFF4CFE6FF1200020EDBCFE9FFDB2A0D
:102D8000030EDBCFEAFF1200DECFE6FFDDCFE6FF6A
:102D9000120058D9A8EF0DF0F3CFDEFFF4CFDDFF1E
:102DA0001200010EDBCF26F0020EDBCF27F0030E60
:102DB000DBCF28F0040EDBCF29F00A0E2B6E2C6A35
:102DC0002D6A2E6AE3EF35F09AD96ED90CD197D9D6
:102DD00063D909D18FD9D89001501200FD0EDBCFF5
:102DE000E9FFFE0EDBCFEAFF1200100EE66EE66A88
:102DF000D80EE66E040EE66E12000DD9090153518D
:102E0000E66EE66A4EC9E6FF4FC9E6FF4CC9E6FF2B
:102E10004DC9E6FF1200E66E5FEC3EF0E55212008F
:102E2000040EDBCF00F0050EDBCF01F0D89001508F
:102E3000120001EC1AF0E552E55205011200E66EAF
:102E40005AEC3AF08FEF18F0006E060EE15E00507B
:102E50001200006E016AD950030FE96EDACFEAFF63
:102E60000050EE260150ED22120031D9040EDB6A2B
:102E7000050EDB6A1200C9EC44F0036E0B0EE15E36
:102E80000350A8EC0DF0DF2A010E1200010EDBCF7B
:102E9000E6FF020EDBCFE6FF120052EC42F0046EBA
:102EA0000A0EE15E04501200FF6FEFEF19F0DECF63
:102EB000E9FFDDCFEAFFCC0EE926080EEA22120078
:102EC000000E005C040E01581200CA0EE66E060EDB
:102ED000E66E120009011351E66EE66A1200D9CFC0
:102EE000E9FFDACFEAFF1200A8EC0DF0A2EF0DF037
:102EF00097EC32F014D9050112003AEC3AF00FD9F0
:102F00000009120096EC39F0036E070EE15E0350E3
:102F100000091200EFD80001800E01141200DF50EA
:102F2000EA6A360FE96E090EEA221200E126FD0E6A
:102F3000DBCFDEFFDBCFDDFF1200DFCFE9FFDF2AD3
:102F4000010EDBCFEAFF1200DECF02F0DDCF03F08F
:102F5000D89003501200D89000360136E8041200D1
:102F6000E10EE66E060EE66E1200E750E926000E50
:102F7000EA221200020EDB2A030E1200C8D844C94E
:102F8000E6FF45C9E6FF46C9E6FF47C9E6FFEED8BA
:102F9000BD0E006E600EB8D8BAD848C9E6FF49C960
:102FA000E6FF4AC9E6FF4BC9E6FFB6EF18F0A7D81F
:102FB000FAEC39F08FEF18F020DE22EF16F0016EF8
:102FC000026A00C0E6FFE66E02C0E6FF1200600E75
:102FD000E66E000EE66E1200E66E2DDE94EC3AF020
:102FE00059DE1BEF16F0E66E9BEC3DF0006E080E0E
:102FF000E15E005012008BD8C9EF44F096DEC40E9B
:10300000006E880E1200A0D8000EE66E060E28DEB6
:10301000DF2A010E120000C0E6FF01C0E6FF120029
:10302000FFDD070EE15E03501200F0DD070EE15EEA
:1030300005501200E8DD2C081200E552E552ACDE26
:10304000C4EF16F0C9EC44F0036E070EE15E0350C6
:10305000120045DE020EE1261200E66EA3EC3FF000
:10306000E552DE5299DEDD521200C7DD92DE020E1D
:103070001200CFEC43F0E552E552120016DEF35099
:10308000E66E1200C8DE93EF0DF0020EE66EA3ECC2
:103090003FF0E552CCEF16F0000EE66E020EE66E43
:1030A000FA0EE66E040E1200000EE66E010EE66EDB
:1030B000F80EE66E040E1200010EE76E8FDE55DF8D
:1030C000EF501200EF6AF1DD67DE8AEF17F0E66E6F
:1030D000F2EC3CF0006E080EE15E00501200020EB1
:1030E000DBCFE9FF030EDBCFEAFF1200E552E7CFAB
:1030F000D9FF1200DECF00F0DDCF01F01200000E8C
:10310000E66E060EE66E120078DD14EF16F0000E85
:10311000E66E050EE66E120073DDA8EF0DF0E552C7
:10312000E552E552E5521200370E006E610E47DFA0
:1031300090DD14EF16F0E66E000EE66E030EE66EFE
:10314000FC0EE66E040E12000601006B010EE66E28
:10315000E66A120087DDB90E026E600E15EF18F0F8
:1031600091DF980E006E5F0EDCEF17F07DEC3EF005
:063170006BDE00EF16F01B
:0A317600D8CFE4FFE0CFE4FFE46EE1
:10318000DACFE4FFE2CFDAFFE9CFE4FFEACFE4FFF2
:10319000F6CFE4FFF7CFE4FFF5CFE4FFF3CFE4FF92
:1031A000F4CFE4FFFACFE4FF00EE20F0140EE804C1
:1031B00003E3EECFE4FFFBD700EE00F0200EE804BF
:1031C00003E3EECFE4FFFBD7E652E5EC41F044EC3D
:1031D00043F0E55200EE1FF0200EE80403E3E5CFD4
:1031E000EDFFFBD700EE33F0140EE80403E3E5CF68
:1031F000EDFFFBD7E5CFFAFFE5CFF4FFE5CFF3FF17
:10320000E5CFF5FFE5CFF7FFE5CFF6FFE5CFEAFF26
:10321000E5CFE9FFE5CFDAFFE550E5CFE0FFE5CF09
:10322000D8FF10000801009B1200F6EC20F0E652D7
:10323000D9CFE6FFDACFE6FFBBEC41F0E552E5522D
:10324000000901E1C9D0FF0E0701E95D01E088D066
:103250000D0EDF5CEDE0FBEC20F0A9EC20F003E1CB
:10326000015001E1E8073A0EDF5C1EE1060EE85D61
:103270001BE3CDEC20F018E1490E015D15E1500E85
:10328000025D12E1440E035D0FE10701E80533EC36
:1032900020F0EF6A050EE66E070EE66E8FEC20F06A
:1032A000FD0EE96FE86BC4D70A0EDF5CC1E10701D0
:1032B000E80727EC21F0040EE85D70E3CDEC20F088
:1032C0006DE1430E015D6AE14D0E025D67E1540E52
:1032D000035D64E1070EDF6EDF50DF2A33EC20F080
:1032E000EF50220804E00701E851DF5CF5E3DF045A
:1032F00033EC20F0EF6A0701D46B140EE66EE66A39
:10330000070EE66E070EE66ED40EE66E070EE66E4C
:10331000F2EC3AF0006E060EE15E00500701E76B3A
:10332000E8C7DFFFDF50DF0633EC20F0EF502C085A
:1033300003E0DF500008F6E3DF50016A000F006E83
:10334000070E0122020E0026000E012200C0E6FF39
:1033500001C0E6FF8FEC20F0E86BFE0EE96F68D746
:10336000FE0EE95D1EE10D0EDF5C03E00A0EDF5C80
:1033700007E1E851E82B33EC20F0200EEF6E02D08D
:10338000FBEC20F0A9EC20F003E1015001E1E8079B
:10339000EA07EA5101E04CD727EC21F0A2D9070156
:1033A00018D00D0EDF5C08E0FBEC20F0A9EC20F05B
:1033B00003E1015001E1E807EA070A0EDF5C06E1DC
:1033C000E80727EC21F08DD90701E86BEA5101E00D
:1033D0002FD7E86BE9692CD7E5526FEF20F0C6ECE8
:1033E00020F00EE0080100B1FDD7C6EC20F0E66E3B
:1033F00094EC41F0E5520501FE2B000EFF23EFD7C0
:103400001200F6EC20F0BAEC20F00FE0080100B159
:10341000FDD7BAEC20F0E66E94EC41F0E552FD0EDB
:10342000DB2AFE0EF0E3DB2AEED76FEF20F0F6EC9E
:1034300020F0080100B1FDD7FE0EDBCFE6FF94ECD3
:1034400041F0E5526FEF20F0F6EC20F0040EE1269B
:10345000030EE66EEEEC20F06C0E026E5E0E3FEC9C
:1034600020F00EE0FD0EDBCF00F0FE0EDBCF01F012
:1034700000C001F0006A00500701EE130150EF1385
:10348000690E026E5E0E3FEC20F00BE0FD0EDBCF0E
:1034900028F0FE0EDBCF29F028500701EE1329504B
:1034A000EF13040EE15C02E2E16AE552E16E6FEFB8
:1034B00020F0F6EC20F0020EE126FE0EDBCFC8F77E
:1034C0000701C851230A01E1F9D0010A01E1ECD05A
:1034D000030A01E1D4D0010A01E1BBD0600A01E195
:1034E0009BD0010A6DE0530A5CE0030A51E0010A37
:1034F00046E0160A3EE0030A33E0010A2AE0070A22
:1035000015E0010A11E0030A01E0E3D00A0E0AEC1B
:1035100021F00701030ECD6F140ECE6FCF6B0901A2
:103520005B6B8CEC0DF0D5D0CD6BD3D0E6682FEC77
:1035300021F0E668E66AD1EC20F038EC43F06FEC5D
:103540003EF00701020ECD6F76EC20F00701CC6B48
:10355000C0D0050ECD6F0A0E76EC20F00A0E6FD0AB
:10356000060ECD6F020ECE6FCF6BC96B6FEC3EF0C7
:10357000B0D0E66A0DEC20F04CEC3EF0AAD0090E7B
:103580000AEC21F099EC20F0DC0EFE6F8A0E89D057
:10359000080E0AEC21F099EC20F0E80EFE6F8A0E7E
:1035A00080D0070E0AEC21F00701030ECD6F230E29
:1035B000CE6FCF6BC96B0501F20EFE6F8A0E71D014
:1035C000050EE66E2FEC21F00701CA07000ECB5B5B
:1035D000D880CA55000ECB5506E2070E5FEC20F0EE
:1035E0000701400E05D0080E5FEC20F00701020E27
:1035F000CD6FCAC7CEF7CBC7CFF70A0ED880CE574C
:10360000000ECF570F0ECF03F3CFCFF7CE03F3CF7C
:10361000CEF7F450CF275DD0050E0AEC21F01BEC5D
:1036200021F022EC20F012E086EC46F000090EE0DA
:103630000701020ECD6F3C0E76EC20F0020E54EC2A
:1036400020F005015D0EFE6F5E0E2BD00701200EEF
:10365000C86F020E0AEC21F00601C96B0701CD6BA1
:10366000C96B0901590507E0050E595D04E0780EA4
:103670000701D26F02D00701D26BD36B2AD0060E9E
:103680000AEC21F0020E54EC20F00701030ECD6F7E
:10369000F00ECE6FCF6B90EC0DF005013F0EFE6F7C
:1036A0008B0E7DEC20F015D0060E0AEC21F0070100
:1036B000230ECD6F1E0ECE6FCF6B0BD0CC51CC2B0B
:1036C000006E140E005C02E2020E01D0030E63ECE9
:1036D00020F0020EE15C02E2E16AE552E16E6FEF7A
:1036E00020F0FE0E0701E95D17E10901590505E02B
:1036F000050E595D02E073EC20F0E8C7E6FF33ECFD
:1037000021F0D40EE66E070EE66E50EC26F0006E49
:10371000050EE15E00501200FF0EE95D0BE033EC98
:1037200021F0FFEC11F0E552E5520A0E0701CA6FD5
:10373000CB6B1200C851200A01E191D1600A01E16E
:10374000ECD0620A01E1CDD0030A01E1ABD0330A2B
:1037500001E17FD0030A52E0010A14E0110A01E0FE
:103760001200020EE85D01E26CD2C2EC20F001E032
:1037700068D24B0E015D01E064D22BEC21F0100EFB
:1037800063EF20F0040EE85D23E3CDEC20F020E1B0
:10379000430E015D1DE1530E025D1AE14D0E035D06
:1037A00017E133EC21F094EC3AF0E552E552F3CF17
:1037B000E9FFF4CFEAFFE906000EEA5A000EE92617
:1037C000070EEA22EF50310818E0030E22EF21F035
:1037D0000701C95101E035D2020EE85D01E231D2A4
:1037E000C2EC20F001E02DD24B0E015D01E029D2A8
:1037F0002BEC21F0110E63EC20F01200080EE85DB6
:1038000012E3CDEC20F00FE1430E015D0CE1500E10
:10381000025D09E1490E035D06E1520E075D18E005
:10382000040E22EF21F00701C95101E00AD2020E75
:10383000E85D01E206D2C2EC20F001E002D24B0EBC
:10384000015D01E0FED12BEC21F0120E63EC20F0C3
:103850001200060EE85D15E3CDEC20F012E1490EF2
:10386000015D0FE1500E025D0CE1520E035D09E1B6
:10387000390E065D06E005016D0EFE6F8B0E7DEFC5
:1038800020F0020E0701E85D01E2DBD1C2EC20F07E
:1038900001E0D7D14B0E015D01E0D3D12BEC21F03B
:1038A000210E53D0020EE85D06E3C2EC20F003E1E6
:1038B0004B0E015D2BE0050E0701E85D07E3450EA9
:1038C0000701005D03E1520E015D09E00A0EE66E9C
:1038D000E66A520E006E5E0E92DB01E0B2D1220E5D
:1038E00034D00DEC21F001E0ACD12C0E0701085DC5
:1038F00003E1070E091502D0070E07150901596FDC
:10390000E80404E0050E595D01E09BD10A0E0701B1
:10391000CA6FCB6BCC6B400E18D0020EE85D17E37C
:10392000450E0701005D13E1520E015D10E1020E2C
:103930000701C95D03E0030EC95D02E1410E05D038
:10394000050EC95D01E08AD0030E63EF20F0020E80
:103950000701E85D06E3C2EC20F003E14B0E015DD8
:103960000BE0530E0701005D03E1480E015D04E02A
:10397000050E0701C95D59E10701E86B1E0ECE6F08
:10398000CF6B09015A6B020E8FDB0701C92BC9519E
:10399000080A49E00F0A3AE0010A33E0030A2CE082
:1039A000010A25E0070A1DE0010A0AE0030A01E016
:1039B00012000501380EFE6F5E0E9FDB050E0CD067
:1039C00005012B0EFE6F5E0E98DB050E15EC21F047
:1039D000060E15EC21F0070E23DB350EFE6F5E0E92
:1039E00020D0040EAFDB1D0EFE6F5E0E1AD0050157
:1039F0000F0EFE6F5E0E15D00501050EFE6F5E0EFA
:103A000010D00501ED0EFE6F5D0E0BD0030E9ADB9C
:103A1000D90EFE6F5D0E71DB040E02DBCF0EFE6F62
:103A20005D0E7DEF20F0200E0CD0070EE85D0BE35D
:103A3000080EE66EE66AC60E006E5D0EE0DA03E181
:103A4000020E63EF20F00B0EE66EE66ABA0E006E11
:103A50005D0ED5DA01E0F5D0020E35DB1200DDDBBC
:103A600024E12C0E0701085D03E1070E091502D0C1
:103A7000070E07150901596FE80403E0050E595DAB
:103A800005E10701D26BD36BE66A0AD00701D25178
:103A9000D31101E0D6D0780ED26FD36B010EE66E53
:103AA000E66A11EC43F0E55255D0050EE66EE66A83
:103AB000B40E006E5D0EA3DA0FE10901590504E0B2
:103AC000050E595D01E00FDB010EEEDA05014E0E29
:103AD000FE6F8B0E7DEF20F00A0EE66EE66AA90EF1
:103AE000006E5D0E8CDA04E109015A511EE113D01B
:103AF000070EE66EE66AA10E006E5D0E80DA2CE11E
:103B0000110EE66EE66A8F0E006E5D0E78DA11E138
:103B100009015A510AE1010EE66EE66E42DB93ECB2
:103B20000DF011EC0EF0A2EC0DF00901010E5A6F30
:103B3000120009015A6B020EE66E91DB090159056C
:103B400004E0050E595D01E07CD090EC0DF0410ED3
:103B5000E66EAFDCE5521200050EE66EE66A890EEF
:103B6000006E5D0E4CDA12E12C0E0701085D09E1D2
:103B7000070E0715006E070E06150A0DF3500024F8
:103B800002D0070E061509015C6F1200070EE66EE3
:103B9000E66A810E006E5D0E32DA08E00B0EE66E0C
:103BA000E66A750E006E5D0E2ADA03E10601C96B46
:103BB0001200090EE66EE66A6B0E006E5D0E1FDAED
:103BC0003CE0060EE66EE66A640E046E5D0E056E5F
:103BD000066A04C0E6FFE66E06C0E6FFF7DA076E87
:103BE000070EE15E0750000928E00A0EE66EE66A5D
:103BF000520E086E5E0E096E0A6A08C0E6FFE66E97
:103C00000AC0E6FFE3DA0B6E070EE15E0B50000917
:103C100014E00B0EE66EE66ABA0E0C6E5D0E0D6ECB
:103C20000E6A0CC0E6FFE66E0EC0E6FFCFDA0F6E3E
:103C3000070EE15E0F50000904E190EC0DF0410E1B
:103C400042DA120045DA40E0220A3CE0230A2EE084
:103C5000330A23E0030A19E0010A0FE0110A01E028
:103C6000EFD0050ECE5D000ECF5902E2020E27DA2C
:103C700005014A0EFE6F8B0E17D098DA01E0E0D0F6
:103C80000501DC0EFE6F8A0E0FD090DA01E0D8D06D
:103C90000501E80EFE6F8A0E07D088DA01E0D0D069
:103CA0000501F20EFE6F8A0E28DACAD0140ECE5D20
:103CB000000ECF5901E3C4D0060EE66EE66A11ECA1
:103CC00043F094D0010E23D0FF0EE95D09E0EB052F
:103CD00003E1EB6BE96910D0EB51010801E2EB075E
:103CE000000ED880D255000ED35508E2D207000E40
:103CF000D35BD251D31102E1210E09D00601C95183
:103D0000000809E2C92BC9513C0805E2400EE66EE5
:103D100059EC1AF06CD00901590504E0050E595D03
:103D200001E08ED00601F951FA1109E00601C8053B
:103D300006E10601C95103E1E8EC12F081D0FF0E63
:103D4000070147DA31E20601C8052EE10A0EACD9B7
:103D5000040E07013EDA06E2EE95F05171E176ECD1
:103D600015F06ED0100E35DA04E2EE99E5EC15F0A0
:103D700067D0020E2EDA04E2EE9392EC0EF060D0E1
:103D8000010E27DA11E2EE9109015B5100080CE205
:103D90000601C95109E10A0E87D993EC0DF052ECE6
:103DA00010F092EC0EF04AD0000E0701EE15006EF6
:103DB000FF0E27DA2EE20A0E77D9C8D9000E0701C6
:103DC000EE15006E040E1DDA07E2EF95F05138E1B2
:103DD0001CDA77EC21F00AD0000EEE15006E100E02
:103DE00010DA07E2EF9911DA38EC22F0E552E552E9
:103DF00027D0000EEE15006E020E03DA02E2EF93FA
:103E000008D0000EEE15006E010EFBD902E2EF9114
:103E100017D009011251000813E20801D45100081B
:103E20000FE20601C9510CE109015B51000808E2EB
:103E3000020E3AD993EC0DF072EC0FF0A2EC0DF0FB
:103E4000020EE15C02E2E16AE552E16E48D107014F
:103E5000C851200A01E012000601C951000802E21F
:103E6000AFEF20F005DA12E0020E1ED90501530E65
:103E7000FE6F8B0EFF6FEFEC19F008014151000847
:103E800003E2010E11D9F9D7020E0ED9120020D982
:103E90001CE10601C951000802E261D916D00901EE
:103EA0005A050FE109015B5100080BE293EC0DF09C
:103EB0000B0EC8D801E0FDD80C0EC4D801E0F9D82B
:103EC0001FD9010E0701C919C96F020EE15C02E298
:103ED000E16AE552E16E03D11200FAD846E1050E1F
:103EE0000901135D27E2800E09010E1523E1070188
:103EF000ED5110E109015A050EE10601C9510BE12E
:103F000093EC0DF0F2EC15F0A2EC0DF00701480E69
:103F1000ED6F01D0ED070701EC510AE117D975D912
:103F200050EC22F0E552E5520701480EEC6F06D046
:103F3000EC0704D00701060EEC6FED6F09015A057E
:103F400014E109015B5111E10601C951000802E2C7
:103F500006D90BD093EC0DF00B0E74D801E0A9D864
:103F60000C0E70D801E0A5D8CBD8020EE15C02E2BD
:103F7000E16AE552E16EB3D00701F051000801E2B9
:103F8000F007D02B000ED123CD5100080DE2EDD863
:103F9000CE07000ECF5B0050011006E1CDC7E6FF53
:103FA00059EC1AF0E55201D04DDEB4D81E0E2D6E3C
:103FB0002E6A06D901E14BDF5BD901E168DFAAD89F
:103FC0002C0E2D6E010E2E6EFBD801E185DFA2D8DE
:103FD000580E2D6E020E2E6EF3D806E17EDF580EBF
:103FE0000701D05F020ED15B12001200800E946EAA
:103FF00078EC41F00901596B010E63EF20F0016E7E
:10400000026A00C0E6FFE66E02C0E6FFDFD8036E7C
:10401000070EE15E03500009120021D92BEF21F0B9
:10402000E66EA3EC3FF0E552F3CF00F0F4CF01F0E1
:10403000F3CFE6FFF4CFE6FF01EC1AF0E552E552CC
:1040400005011200E66ECAD8DECFE9FFDDCFEAFF38
:10405000EF501200D5EC46F024C000F025C001F06E
:10406000245025101200EA6A000FE96E070EEA22BA
:104070001200000ED8800054000E01541200036E8E
:10408000046A02C0E6FFE66E04C0E6FFBED820EC7C
:104090003BF0056E050EE15E0550F3CF00F0F4CF66
:1040A00001F0F350F4101200E66E5FEC3EF0E552C2
:1040B0001200ABD8F6EC10F0E552E5521200E66EB5
:1040C000E66AD1EF20F0E66E59EC1AF0E5521200E4
:1040D0008DD8020EE1260701C851200A1200E552D0
:1040E000E7CFD9FF1200A7D82BEF21F0CE6FCF6B0F
:1040F000C96B09015B6B90EF0DF0FF6FEFEF19F0EB
:1041000092EC0EF072EC0FF08AEC0FF052EC10F023
:10411000A2EF0DF0D0C700F0D1C701F01200CFEC34
:1041200043F0E552E552F3CFEAF707013C0EEB6F9F
:1041300012000701030ECD6F5F0ECE6FCF6BC96B00
:1041400005011200E66E8BD805011200E66AEEEF5B
:1041500020F0E851006E016AC80E00181200050E2A
:104160000701D05F000ED15B1200CEC700F0CFC7B1
:1041700001F01200FD0EDBCFE9FFFE0EDBCFEAFF00
:10418000EF5012004F0E0701005D1200FEC5F6FF52
:10419000FFC5F7FF0800F55012002B0E0701005D68
:1041A000120011EC43F0E552E5521200DEDF030E7F
:1041B0002D6E2E6ACEC728F0CFC729F02AEF20F047
:1041C000D0C728F0D1C729F02AEF20F04CD896EFBD
:1041D00039F0EE15006E016A39EF20F0A3EC3FF0E4
:1041E000E552F3CFDEFFF4CFDDFF1200D9CFE6FFBB
:1041F000E1CFD9FF1200E851E82B35DFDFCFEFFF29
:104200001200EF15016E39EF20F0DECFE6FFDDCFB3
:10421000E6FF1200E66E0DEF20F0050EE66EE66A90
:104220004C0E006E5E0EFFEF1FF0FADE270EFE6FE3
:104230005E0E7DEF20F00701D26BD36B0901050EF6
:10424000596F12003CDF0701010EC96F1200E851DF
:104250000ADFEF6A1200E66AE66AD1EF20F0010E8B
:10426000E66ED1EF20F0000EE66E070EE66E12004D
:0C42700051DF3C0E2D6E2E6AE0EF20F0B6
:04427C0046EC27F0F5
:104280000501DF0EFE6F630E2AEC28F026EC27F006
:104290007DEC28F00501DB0EFE6F630E2AEC28F0A2
:1042A000020EA9EC27F04BEF27F046EC27F00801AF
:1042B000DAB50AD00EEC28F0F9C8FEF5FAC8FFF519
:1042C000EFEC19F055EC27F04BEF27F046EC27F018
:1042D0000801DAB50AD00EEC28F0FBC8E6FFFCC8EE
:1042E000E6FF7DEC28F055EC27F04BEF27F00AECC9
:1042F00028F00801DAB5B4D0A9EC27F00EEC28F0CC
:1043000009010EA54AD009010B51040A15E0070A5C
:104310000EE0020A07E0010A16E10501CD0EFE6F6C
:10432000630E0ED00501C20EFE6F630E09D00501AB
:10433000B90EFE6F630E04D00501AA0EFE6F630E68
:10434000FF6FEFEC19F0090109510F0A21E0020A91
:104350001AE0090A13E0060A0CE0030A05E0050169
:10436000460EFE6F630E1DD00501A10EFE6F630E9B
:1043700018D005018B0EFE6F630E13D005017D0E64
:10438000FE6F630E0ED00501690EFE6F630E09D03D
:104390000501570EFE6F630E04D00501390EFE6F46
:1043A000630E2AEC28F00501290EFE6F630E2AEC3D
:1043B00028F0020EE66E4FEC28F066EC27F04D0870
:1043C0000DE114C9E6FF15C9E6FF230E006E630E6A
:1043D000E5EC27F0070EE15E035031D014C900F080
:1043E00015C901F0040ED89000360136E804FBE14F
:1043F000050E0026000E01220A0E2D6E2E6A00C048
:1044000028F001C029F0D5EC46F028C000F029C002
:1044100001F028C0E6FF29C0E6FF1D0E026E630E04
:10442000036E046A02C0E6FFE66E04C0E6FF82EC9B
:1044300028F0C9EC44F0056E070EE15E055007EC6C
:1044400028F00501150EFE6F630E2AEC28F0090115
:104450001351E66EE66A100E006E630E3FEC28F014
:10446000020EE15C02E2E16AE552E16E4BEF27F0F9
:104470000AEC28F00801DAB50BD0A9EC27F072ECB1
:1044800028F08D0EFE6F6F0E2AEC28F055EC27F009
:10449000020EE15C02E2E16AE552E16E4BEF27F0C9
:1044A0000AEC28F00A0EA9EC27F00EEC28F009011E
:1044B0001351E66EE66ADE0E006E620E3FEC28F0E7
:1044C000050EA9EC27F0020EE15C02E2E16AE5527A
:1044D000E16E4BEF27F00AEC28F0E66A34EC27F0A7
:1044E000A1EC27F026EC27F0AEEC27F002E1010E5C
:1044F00006D00801DAB302D095EC28F0000E006E69
:10450000020EE15C02E2E16AE552E16E00504BEF1F
:1045100027F00AEC28F0010E3CEC28F0A1EC27F083
:104520008DEC27F0AEEC27F002E1010E06D0080179
:10453000DAB302D095EC28F0000E006E020EE15CBA
:1045400002E2E16AE552E16E00504BEF27F00AEC1F
:1045500028F05AEC28F000C0E6FF01C0E6FF26EC88
:1045600027F094EC3AF04BEC28F0E7CF01F0E5525D
:10457000E7CF00F00050F3240801F76F0150F4205A
:10458000F86FF7C800F0016EFD0EDB50001807E170
:10459000FE0EDB50011803E1F36AF46A16D0FD0E3B
:1045A000D6EC27F057EC28F008E066EC27F005E0A1
:1045B000DF2A010EF7E3DB2AF5D757EC28F003E1F9
:1045C00042EC28F0EF6AC6EC27F0020EE15C02E252
:1045D000E16AE552E16E4BEF27F00AEC28F0FD0EA0
:1045E000D6EC27F066EC27F005E0DF2A010EFAE3AF
:1045F000DB2AF8D7DECF00F0DDCF01F00801F7515C
:10460000001806E1F851011803E1F36AF46A21D0B9
:10461000DF2A010E01E3DB2AD9CFE9FFDACFEAFF77
:10462000FD0EEECFDBFFFE0EEDCFDBFF57EC28F0EB
:1046300008E066EC27F005E0DF2A010EF7E3DB2A4D
:10464000F5D757EC28F003E142EC28F0EF6AC6EC0E
:1046500027F0020EE15C02E2E16AE552E16E4BEF07
:1046600027F09BEC28F003E0EBEC27F003E1EFEC04
:1046700027F00BE0E66A34EC27F0C80E006E620EFD
:10468000E5EC27F0070E15EC28F0020EE15C02E2E3
:10469000E16AE552E16E4BEF27F046EC27F0EBECD8
:1046A00027F00CE0D3DBE66AE8EC3FF04BEC28F0B7
:1046B0000801500EF96F6E0EF2EC27F0ECD39BEC74
:1046C00028F003E0EBEC27F003E1EFEC27F00BE040
:1046D000010E3CEC28F0B40E006E620EE5EC27F003
:1046E000070E15EC28F0020EE15C02E2E16AE552E9
:1046F000E16ED1D36FEC28F009E0AFDB010EDBDB1C
:1047000008017D0EF96F6E0EF2EC27F0C4D336EC83
:1047100028F003E0EBEC27F003E1EFEC27F028E0D2
:104720000801DAB525D0020EA9EC27F072EC28F0CA
:10473000B10EFE6F6F0ED3EC27F044C9E6FF45C9FA
:10474000E6FF46C9E6FF47C9E6FF75EC28F005011C
:10475000B20EFE6F620ED3EC27F048C9E6FF49C9DE
:10476000E6FF4AC9E6FF4BC9E6FF75EC28F09DDB82
:1047700092D336EC28F003E0EBEC27F003E1EFEC0A
:1047800027F004E063DBB3DDE552E55284D37EDB42
:10479000030EE12672DB03E0EBEC27F003E1EFEC24
:1047A00027F033E00801DAB530D072EC28F0AA0E19
:1047B000FE6F620E2AEC28F0DF6A200EDF5C24E236
:1047C000DFCFE6FFA3EC3FF0E552DE52F3CFDEFF92
:1047D000F4CFDDFFDD52010EDBCFE9FF020EDBCFB0
:1047E000EAFFEF500FE0DFCFE6FFE66AA40E006EAF
:1047F000620E26DB010EDBCFE6FF020EDBCFE6FF0B
:104800007DEC28F0DF2AD9D750DB030EE15C02E211
:10481000E16AE552E16E3FD339DBE652020EDF6E0C
:10482000DEDB1EE039EC28F01BE0200EDF5C12E23C
:104830002DEC28F00FE021DB2D0804E160DB02E124
:1048400048DB01D00ADBDF50DF2A35DB06DB1FEC5B
:1048500028F0EBD708019F0EF96F6E0EC3DB8ADBE1
:10486000E55219D39EEC28F004E107DB1EE0B3DB30
:104870001CE00801DAB519D072EC28F09C0EFE6F2E
:10488000620EE8DB080E3CEC28F08D0E006E620E26
:10489000D7DA020EF1DB820E006E620ED1DA030E61
:1048A000EBDB6F0E006E620EEADB020EE15C02E2F1
:1048B000E16AE552E16EEFD26FEC28F013E0D9DB4C
:1048C00011E0CBDA080EADDB07E0C7DA020EA9DB98
:1048D00003E0C3DA030EEFDA8DDBC4DF71DBA7EC94
:1048E0003BF048DBD8D29EEC28F004E1C6DA33E096
:1048F00072DB31E00801DAB52ED0F4DB690EFE6F11
:10490000620EA8DB050EB8DB600E006E620E98DA50
:10491000060EB2DB560E006E620E92DA070E87ECC0
:1049200028F00601C85105E00501270EFE6F620E52
:1049300008D0200E0701C85D06E10501060EFE6FD6
:10494000620E88DB07D0C851E66EE66AE30E006EA1
:10495000610E76DAAADA020EE15C02E2E16AE55261
:10496000E16E99D2BCDB1FE084DB1DE076DA050E38
:1049700058DB15E082DA2D0804E1C1DA02E1A9DA98
:1049800001D06BDA060E4DDB0AE077DA2D0804E180
:10499000B6DA02E19EDA01D060DA070E8CDA2ADBA1
:1049A000A2DF0EDBE7DA77D2C9DB04E166DA18E0D2
:1049B00012DB16E00801DAB513D094DBDB0EFE6FD4
:1049C000610E48DB040E58DBD30E006E610E38DA40
:1049D000090E9DDB0A0E50DBC50E006E610E4FDB2B
:1049E000020EE15C02E2E16AE552E16E54D277DB4D
:1049F00011E03FDB0FE031DA040E13DB07E02DDAC4
:104A0000090E0FDB03E029DA0A0E55DAF3DACCDF00
:104A1000D7DAB0DA40D22ADB02E0DDDA02E1DFDA0F
:104A200020E00801DAB51DD05DDBBF0EFE6F610E20
:104A300011DB0601FB51E66EE66AB20E006E610EF6
:104A4000FFD90601FC51E66EE66AA50E006E610E06
:104A5000F7D90701C851E66EE66A920E006E610E44
:104A60000EDB19D213DAE65208DA02E0B4DA02E118
:104A7000B6DA21E00801DAB51ED034DB880EFE6F0D
:104A8000610EE8DADF6A100EDF5C14E285DAEF50BF
:104A90000FE082DAEF50E66EE66ADFCFE6FFE66A05
:104AA000800E006E610E91DA090EE15E0350AFDAFE
:104AB000DF2AE9D7FAD9E552EED1E8D9E6528FDA02
:104AC00026E0D7DA24E0C9D95BDADF6EC6D9B7DAD7
:104AD000000EDF5C1CE3100EDF5C19E2BEDA17E0AB
:104AE000D6DA5ADAE552E750EF6E080EDF5C05E3DE
:104AF000B4D9080EDF5C180FDED90F0EDF5C02E1BF
:104B0000A7EC3BF00801B90EF96F6E0E6BDAE552B7
:104B1000C2D1E5DA09E0BBDAC8EC3CF0E5520801A5
:104B2000CF0EF96F6E0E5EDAB6D1D9DA08E095D9FC
:104B3000020EE66E01DAE20EF96F6E0E53DAABD1B9
:104B4000CEDA08E08AD9030EE66EF6D9F90EF96FCF
:104B50006E0E48DAA0D1C3DA07E07FD9E66AECD955
:104B6000120EF96F6F0E3EDA96D1B9DA08E075D9F8
:104B7000010EE66EE1D9270EF96F6F0E33DA8BD195
:104B8000AEDA3EE076DA3CE068D943EC3BF0E55241
:104B9000E552030EE66EE66A7C0E006E610E26DAC2
:104BA00002E1E66A1ED0030EE66EE66A780E006E3B
:104BB000610E1CDA02E1010E13D0030EE66EE66A06
:104BC000740E006E610E12DA02E1030E09D0030EBC
:104BD000E66EE66A700E006E610E08DA11E1040EF0
:104BE000E66EC3EC3CF0E55238D944D904E04FDA24
:104BF000C4EC3CF0E5520801430EF96F6F0EF2D998
:104C00004AD134DA02E0E7D902E1E9D90CE0010E39
:104C1000E66EC5EC3CF0E5520701F06B0801600E52
:104C2000F96F6F0EDFD937D121DA02E0D4D902E172
:104C3000D6D90CE0E66AC5EC3CF0E55207011E0E41
:104C4000F06F0801770EF96F6F0ECCD924D10EDA10
:104C500002E0C1D902E1C3D910E009010251E66EB8
:104C6000E66A0151E66EE66A0051E66EE66A500EAB
:104C7000006E610EAAD90B0ED8D90DD15CDA02E014
:104C8000AAD902E1ACD905E0030EE66E59EC1AF0A0
:104C9000E552020EE15C02E2E16AE552E16EFBD010
:104CA000F5D8040EE126FB0E81D910D917E0FFD903
:104CB00015E00CD960080DE2E5D9EFCF00F07B0ECE
:104CC000005C07E203D9E00FE66EDCD9E552E7505D
:104CD000EF6EDF2A010EE9E3DB2AE7D7E8D904E12A
:104CE000DF2A010E01E3DB2A020EDB6A030EDB6A18
:104CF000020EDBCFF6FF030EDBCFF7FF1B0EF70232
:104D0000F3CFF7FFF602F3CFF6FFF450F726370E96
:104D1000F626700EF7220800F55001E184D0020E4D
:104D2000DBCF02F0030EDBCF03F01B0E0302F3CF49
:104D300003F00202F3CF02F0F4500326370E0226EE
:104D4000700E0322046A02C0E6FF03C0E6FF04C03F
:104D5000E6FFA2EC3AF09FD927C000F028C001F08E
:104D600027C0E6FF28C0E6FF020EDBCF05F0030EEA
:104D7000DBCF06F01B0E0602F3CF06F00502F3CFE1
:104D800005F0F4500626370E0526700E0622076A37
:104D900005C0E6FF06C0E6FF07C0E6FFBED896ECFA
:104DA00039F0086E070EE15E0850000935E1020E89
:104DB000DBCFE9FF030EDBCFEAFFD890E936EA3616
:104DC000C80EE926050EEA22EECF00F0EFCF01F083
:104DD000DECFE6FFDDCFE6FFFB0EDBCFE6FFFC0E0E
:104DE000DBCFE6FFFA0EDBCFE6FFFB0EDBCFE6FF05
:104DF000FC0EDBCFE6FFFD0EDBCFE6FFFE0EDBCFCA
:104E0000E6FF04D001C0FAFF0050F96EFBDF026E2E
:104E1000090EE15E02500DD0020EDB2A030E01E204
:104E200067D7DB2A65D779D811D850EC15F033D97C
:104E3000E552040EE15C02E2E16AE552E16E2BD03C
:104E4000C4D8070EE15E035007EF28F0FD0EDBCF5C
:104E5000E6FFFE0EDBCFE6FF1200F60EDBCFE6FF2D
:104E6000F70EDBCFE6FF12001AD9DECFE6FFDDCF6B
:104E7000E6FF1200E4D82DEF28F023D9EF501200FE
:104E80006BEC22F0E552E55200091200D9CFE6FFA3
:104E9000E1CFD9FF1200E552E7CFD9FF120089EC2C
:104EA00022F0F9D8E552000912000501D90EFE6F73
:104EB000630E2AEF28F0E66EE8EC3FF04BEF28F0A7
:104EC000A7EC22F005D9F350F4101200DBD8EF5014
:104ED0001200010EE76EF60EDBCF00F0F70EDBCF0F
:104EE00001F0E7500026000E012200C0E6FF01C0DD
:104EF000E6FF120055EC21F0E552E5521200010EDA
:104F0000E76EDFD8E750E926000EEA22EF501200E4
:104F10003EEC21F0E552E5521200FB0EDBCFE6FF3E
:104F2000FC0EDBCFE6FF120096EC39F0036E070EA5
:104F3000E15E035000091200C6EC3CF0ACD8080159
:104F4000120094EC3AF0C4D8F3CFE6FFF4CFE6FFBA
:104F50001200E66E5FEC3EF0E5521200DECFE6FF97
:104F6000DDCFE6FFC7EC3AF0026E060EE15E0250BE
:104F700000091200400EE66E59EC1AF0E5521200DC
:104F8000CFEC43F0E552E552F350120093D800C045
:104F9000F3FF01C0F4FF1200DF50EA6ACC0FE96EA4
:104FA000080EEA22120056D882EF28F0DBCFDEFF8F
:104FB000DBCFDDFF120066EC21F0E552E552120076
:104FC000006E090EE15E00501200A7D89BD8C9EC14
:104FD00044F0036E120041DF39DF4FEF27F036DF78
:104FE00040EF27F0FA6F32DF7AEF27F096D835DFFF
:104FF00094EF27F032DFF80EDBCFE6FFF90EDBCFC0
:10500000E6FFFA0EDBCFE6FF88DF26EF27F07AD83F
:105010007DEF28F03BDF020EE126120017DF88EF5C
:1050200027F049DF1ADF3AEF27F0E15E035008016D
:10503000000EFB6F060EFC6F09DFDBEF27F0EDECD7
:1050400022F0E552E552F60EF3CFDBFFF70EF4CF78
:10505000DBFF1200FF6FEFEF19F0D950F60FE96E8A
:10506000FF0EDA20EA6EEE50ED1012000FDF3DEF7A
:1050700027F0F3DE60EF27F0E66E34EF27F0E0DE96
:1050800055EF27F0DECFE9FFDDCFEAFF1200E5DEC6
:1050900077DFE66E1200E552E552E5521200A3EC0E
:1050A0003FF0E552F3CFDEFFF4CFDDFF12000EDF5D
:1050B00020081200FD0EDBCF00F0FE0EDBCF01F06A
:1050C0001200F60EDBCFE9FFF70EDBCFEAFF12008E
:1050D000E552E552F3CF00F0F4CF01F01200D6DE36
:1050E000EFEF27F09BDF050112007DEC3EF0006E34
:1050F000060EE15E005007EF28F001EC1AF0E552D1
:10510000E5521200000EE66E060EE66E1200B4DFE7
:10511000480E006E620E20EF27F0016E026A00C09A
:10512000E6FFE66E02C0E6FF120008013E0EF96FD0
:105130006E0EF2EF27F06EDF3DEF27F06BDFEFEF43
:0251400027F056
:0E514200DDEC2DF0FB0EDBCFF3FFDB06F350B0
:1051500000090AE02BEC2EF0FA0E96EC2EF0F3E1AB
:10516000011CF1E1010E01D0000E0CEF2EF0DDEC80
:105170002DF03B0EE12402E3E168E652E16E010E00
:10518000DB6A020EDB6AF90EDBCFF6FFFA0EDBCF2D
:10519000F7FFFB0EDBCFF8FF0800F550DF6EDF50A6
:1051A00002E130EF2DF0250EDF5C02E023EF2DF061
:1051B000030EDB6A040EDB6A050EDB6A060EDB6A91
:1051C000070EDB6A45EC2DF02D0EDF5C0CE02B0E9C
:1051D000DF5C09E0200EDF5C06E0230EDF5C03E00D
:1051E000300EDF5C1AE1DF50300A14E0130A0FE0E2
:1051F000030A0AE00B0A05E0060AE4E1030EDB807D
:10520000E1D7030EDB82DED7030EDB84DBD7030E90
:10521000DB86D8D7030EDB88D5D72A0EDF5C1BE1EF
:1052200041EC2DF08FEC2DF010E0030EDB802868B0
:105230002968130EDBCF2DF0140EDBCF2EF0F2EC2D
:1052400036F0040E26C0DBFF03D0130E78EC2DF0F1
:1052500045EC2DF00BD0090EDB6AE6EC2DF003E0F7
:105260005AEC2EF0FAD7090E78EC2DF0030EDBB0D5
:10527000DB982E0EDF5C1BE145EC2DF02A0EDF5C87
:105280000BE141EC2DF08FEC2DF003E1130ECAEC95
:105290002DF045EC2DF00BD0090EDB6AE6EC2DF07D
:1052A00003E05AEC2EF0FAD7090ECAEC2DF0680E86
:1052B000DF5C07E145EC2DF0680EDF5C1DE1030EBD
:1052C00018D0740EDF5C17E07A0EDF5C14E0480E35
:1052D000DF5C06E0540EDF5C03E05A0EDF5C02E1A7
:1052E000020E07D06C0EDF5C03E06A0EDF5C04E1A7
:1052F000010E1DEC2EF0C9DBDF506E0A01E17FD3F9
:105300001E0A01E192D1200A01E18FD13F0A01E199
:1053100049D11A0A01E146D10D0A01E143D1200A1F
:1053200001E140D13A0A01E13DD1200A01E13AD13F
:10533000260A01E135D10D0A01E132D11A0A01E153
:10534000D9D0200A4AE0300A1FE0460A0EE0250ABA
:1053500001E083D3D950F90FE96EFF0EDA20EA6E2F
:10536000010EEE5E000EEE5AEE5A2BEC2EF0250EDC
:10537000E66E95DB03E1011C01E169D327EC2EF019
:1053800001E26BD3DB2A69D3080EDB6A040EDB5023
:10539000010806E2040EDB04EFEC2DF0DB508BDBA2
:1053A000080EDB5009E0030EDB50010B05E172DB58
:1053B00001E04DD3080EDB6A64DBEFCFDFFF9FEC2B
:1053C0002EF003E1011C01E142D327EC2EF001E3B2
:1053D000DB2A60DB01E141D33AD3070EDB50020840
:1053E0000FE16BEC2EF0030E32EC2EF00E0EEECF32
:1053F000DBFF0F0EEECFDBFF100EEECFDBFF20D07A
:10540000F70EDBCF03F0F80EDBCF04F0020E035EE5
:10541000000E045AF70E03C0DBFFF80E04C0DBFFDA
:1054200003C0E9FF04C0EAFF22EC2EF0026A0E0E70
:1054300000C0DBFF0F0E01C0DBFF100E02C0DBFF60
:105440000E0EDBCFE6FF0F0EDBCFE6FF100EDBCF3D
:10545000E6FFA2EC3AF0E552E552E552130E27C002
:10546000DBFF140E28C0DBFF060EDB5005E0130E39
:1054700066EC2EF001E26ADB8AEC2EF002E2130EFB
:1054800037DB4DEC2EF006E0040E66EC2EF002E267
:10549000050E2EDB030EDBB005D0FCDA01E0D7D21F
:1054A000080EDB6A090EDB6A0E0EDBCFF6FF0F0E6D
:1054B000DBCFF7FF100EDBCFF8FF0800F550DF6EF3
:1054C000DF5014E090EC2EF011E29FEC2EF003E19F
:1054D000011C01E1BCD2BBDB01E3DB2A090EDB2AA4
:1054E000D9500E0FE96E000ECBDBE7D7D3DA01E11E
:1054F000B4D2ADD2C6DA110EEECFDBFF120EEDCF75
:10550000DBFF110EDBCFE6FF120EDBCFE6FF94ECE4
:105510003AF0E552E552130EF3CFDBFF140EF4CF51
:10552000DBFF060EDB5004E0130ED0DB01E20EDBE6
:105530008AEC2EF002E2130EDBDAAFDB05E0040E9C
:10554000C5DB02E2050ED4DA030EDBB005D0A2DA29
:1055500001E07DD2080EDB6A090EDB6A110EDBCF9B
:10556000E9FF120EDBCFEAFFEFCFDFFFDF5014E0E1
:10557000D7DB12E2E4DB03E1011C01E168D267DB67
:1055800001E3DB2A090EDB2A110EDB2ADBCFE9FF60
:10559000120EE8E3DB2AE6D77DDA01E15ED257D2CC
:1055A000030EDB8E070EDB0410E195DB040E5ADBE5
:1055B0000A0EEECFDBFF0B0EEECFDBFF0C0EEECFB5
:1055C000DBFF0D0EEECFDBFF6CD0070EDB500308C8
:1055D0002CE1030EDBAE0DD0B2DA020E76DAEFCF9D
:1055E00000F0016A026A036A00AE39D001680268FD
:1055F00035D0F70EDBCF01F0F80EDBCF02F0020E54
:10560000015E000E025AF70E01C0DBFFF80E02C069
:10561000DBFF01C0E9FF02C0EAFFEFCF00F00A0E96
:1056200000C0DBFF0B0EDB6A38D0070EDB50020830
:1056300009E1030EDBAE04D059DB02AE10D00ED070
:1056400055DB0DD0030EDBAE12D079DA020E3DDA57
:10565000F9DA026A036A01AE02D002680368E2DA8C
:105660000C0E02C0DBFF0D0E03C0DBFF1AD0F70EDD
:10567000DBCF02F0F80EDBCF03F0020E025E000E6D
:10568000035AF70E02C0DBFFF80E03C0DBFF02C0B7
:10569000E9FF03C0EAFFD6DAC5DA0C0EDB6A0D0EAD
:1056A000DB6A060EDB5005E1010EF36E050EF3CF4B
:1056B000DBFF150EDB6A160EDB6AD950370F006E62
:1056C000000EDA20016E390E00C0DBFF3A0E01C079
:1056D000DBFF380EDB6A080EDB6A0A0EAEDADF503B
:1056E000780A12E0200A10E0280A0CE0200A0AE0FA
:1056F0003F0A06E00D0A02E0200A08E1020E05D08A
:10570000080E03D0080EDF26100E97DA030EDBBE5C
:1057100002D0DB92DB94DB50800B24E08ADAD89055
:10572000030EEB50000A08E6000EEE5C000EEE5889
:10573000000EEE58000EEE5815E213DA2B682C68B6
:105740002D682E6848EC46F00A0E22C0DBFF0B0ED7
:1057500023C0DBFF0C0E24C0DBFF0D0E25C0DBFFDA
:105760002D0E08D0030EDBA202D02B0E03D0DBA43B
:1057700008D0200EF36E170EF3CFDBFF150EDB2AD9
:1057800002D0170EDB6A050EDB5003E1B7D901E149
:1057900089D06E0E006E8E0E016E000E026E070E28
:1057A000DBCF03F0046A056A066A03C02BF004C06D
:1057B0002CF005C02DF006C02EF0D3D9B1EC46F088
:1057C00000502224F36E01502320F46E0250242056
:1057D000F86EF4CFF7FFF3CFF6FF0800090EF5CF10
:1057E000DBFF580EDF5C0FE1610EF36E090E7BD913
:1057F0000AE3200E006E090EDBCFE7FF0050E75EE4
:10580000090EE7CFDBFF070EDBCF00F0016A026A6B
:10581000036A0FDA00C02BF001C02CF002C02DF09B
:1058200003C02EF0EECF26F0EECF27F0EECF28F01B
:10583000EFCF29F0B1EC46F029C0EDFF28C0EDFF15
:1058400027C0EDFF26C0EFFF390EDBCFE9FFDB06F7
:105850003A0EDBCFEAFF01E2DB06090EDBCFEFFFFA
:10586000150EDB2A4BD995E1030EDBA61DD06F0E7A
:10587000DF5C06E1C1D918E3150EDB285BDA14D032
:10588000780EDF5C09E0580EDF5C06E0620EDF5C3C
:1058900003E0420EDF5C08E1020EF36E160EF3CF5A
:1058A000DBFF02D0150EDB6A030EDB50100B0EE09F
:1058B000040EDBCF00F0050EDB50D880005406E26A
:1058C000060EDB5003E1040EDB5034DA95D90AE210
:1058D000050EDBCFE7FF150EDB50E75E050EE7CFC9
:1058E000DBFF02D0050EDB6A040EDBCF00F0160EE4
:1058F00045D9D880005414E2160EDBCFE6FF150E12
:10590000DBCFE6FF040EDBCFE6FF050EDB50E552F2
:10591000E75CE552D880E754E552D880E7545FD978
:10592000030EDB50010B0BE1080EDB5008E0B2D890
:1059300001E08DD0080EDB50BED8080EDB6A170ED2
:10594000DB5007E088D9170EF1D903E1011C01E112
:105950007ED0160EDB5016E07ED9300EE66E9FD854
:1059600002E1011C74E077D9DFCFE6FF06EC46F0D8
:10597000E552E552E552F4CF01F00001F31C02E1DB
:10598000011C65E0050EDBCF00F0160EDB50D88061
:10599000005409E2050EDBCFE7FF160EDB50E75E91
:1059A000050EE7CFDBFF300EE66E050ECBD94FE1DB
:1059B000390EDB2ADBCFE9FF3A0E01E3DB2ADBCF2E
:1059C000EAFF090EEFCFDBFFDB500EE044D9090EF2
:1059D000ADD902E1011C3BE0390EDB2ADBCFE9FF48
:1059E0003A0EEDE3DB2AEBD755D831E1160EDBCFCB
:1059F000E6FF080EC3D8E552E7245DD82ED0070E87
:105A0000DB50030A1CE0010A14E0030A07E07BD91B
:105A1000DBCFEEFF020EDBCFEDFF1FD0F5D8056A1E
:105A200003AE02D0046805682CD8BCD805C0EEFFD0
:105A300014D0EAD803BE046824D8B4D80ED063D9F1
:105A4000DBCFEFFF0AD07BD905E1011C03E1F3684E
:105A5000F46810D0FCD801E3DB2A79D9CCEF28F028
:105A6000010EDBCF00F0020EDBCF01F000C0F3FF30
:105A700001C0F4FF3B0EE15C02E2E16AE552E16E37
:105A8000CBD029D9020E32EF2EF061D90800F550A3
:105A9000DF6E1200200EE66E080EA2EF2EF006EC6E
:105AA00046F0E552E552E552F3CF00F0F4CF01F0B5
:105AB0000001F31C1200006E016AD950010F4DD98C
:105AC0000050EE260150ED221200045E000E055A31
:105AD000F70E04C0DBFFF80E05C0DBFF04C0E9FFD2
:105AE00005C0EAFF1200DBCFF4FFF350F45C1200B4
:105AF000DB50E76E040EE7CFDBFF12000A0EDBCFB0
:105B000000F00B0EDBCF01F00C0EDBCF02F00D0E20
:105B1000DBCF03F000500110021003101200130E2F
:105B2000EECFDBFF140EEDCFDBFF130EDBCF00F06B
:105B3000140EDBCF01F00001800E01141200F70EED
:105B4000DBCF04F0F80EDBCF05F01200050EDB50C2
:105B5000E66ED950130F01D9E552E750EE6EED6AAB
:105B600012000A0EDBCF26F00B0EDBCF27F00C0E57
:105B7000DBCF28F00D0EDBCF29F01200DBCFE6FFE4
:105B8000150EDBCFE6FF050EDB50E552E724E552AC
:105B9000E7241200DB50CED8010EF36E060EF3CFD1
:105BA000DBFF1200EE50EFCFEAFFE96E02C0EEFF1E
:105BB00003C0EEFF04C0EEFF1200D9CFE6FFDACF3C
:105BC000E6FFE1CFD9FFE2CFDAFF1200DFCFE6FF39
:105BD000E66AEBEC46F0E552E552F3501200E76E50
:105BE000080EE7CFDBFF1200EECF00F0EECF01F0A2
:105BF000EFCF02F0036A1200050EDBCF00F0150EA6
:105C0000DB50D88000541200010EDBCF02F0020EF0
:105C1000DBCF03F0046A1200E552E5CFDAFFE7CFED
:105C2000D9FF12000A0E00C0DBFF0B0E01C0DBFF24
:105C30001200D9500A0FADEF2EF0F36E070EF3CF1E
:105C4000DBFF1200EECF00F0EFCF01F01200010EEB
:105C5000DB2A020E1200FC0EDBCFE6FFFD0EDBCFCF
:105C6000E6FF1200005E000E015AF70E00C0DBFFD7
:105C7000F80E01C0DBFF00C0E9FF01C0EAFF12001F
:105C8000DA20EA6EEF2AEECFF6FF000EEF22EECF1B
:105C9000F7FFEF22EECFF8FF1200040EDBCFE6FF96
:105CA000130EDB50E552E75C9ADFDB5004DF060E93
:105CB000DB501200090EDB500A0DF350DF24D00F29
:105CC000E76E090EE7CFDBFF45EF2DF0DB50F36EFB
:105CD000050E73EF2DF0F70EDBCF00F0F80EDBCFE3
:105CE00001F01200DFCFE6FF4FEF2DF028DF030EAB
:105CF000ECDEF4EF2DF0A1EC28F0E552E552E55290
:105D0000E55200091200BDDEEE50EFCFEAFFE96E6A
:105D1000010E1200130EDB50F36E040E73EF2DF024
:105D2000040EDB50F36E090E73EF2DF0DBCFE6FFB0
:105D30004FEF2DF0E76E050EE7CFDBFF12008BDF94
:105D400072EF2EF0DBCFE6FF86DF7BEF2EF0D9502F
:105D5000F90FE96EFF0E40EF2EF0E96E000EDA202B
:045D6000EA6E1200D5
:0C5D6400434C4F5345440053454E44202F
:105D70004641494C0044415441204143434550541D
:105D80000053454E44204F4B002B4353513A005390
:105D9000544154453A20434F4E4E454354204F4BB7
:105DA0000053544154453A2000434F4E4E4543540E
:105DB000204F4B002B434C4950002B5044503A206D
:105DC0004445414354002B435245473A203000227A
:105DD0002C2236383637220D0041542B434950537C
:105DE000544152543D22544350222C220041542B02
:105DF000434C504F52543D22544350222C223638AB
:105E00003637220D0041542B43494653520D004171
:105E1000542B434950484541443D310D0041542BDA
:105E200043494943520D00222C220041542B435335
:105E300054543D2200220D0041542B434744434F0C
:105E40004E543D312C224950222C22002B435245E6
:105E500047002B434D45204552524F520041542B91
:105E6000434950534855540D00495000534D530079
:105E70004D502D30205041414C455254212121207C
:105E8000435249544943414C20534F43204C4556BB
:105E9000454C20415050524F41434845442028250D
:105EA00075252520534F4329004D502D302050415A
:105EB0005472756E6B20686173206265656E206F29
:105EC00070656E6564202876616C6574206D6F6402
:105ED00065292E00257525250020534F433A2000C3
:105EE0002575204B6D002575206D69000D49646591
:105EF000616C2052616E67653A2000436861726789
:105F0000696E672053746F707065640043686172D6
:105F100067696E672C2048656174696E670050720E
:105F200065706172696E67004368617267696E6768
:105F300020446F6E65004368617267696E672C204C
:105F4000546F7070696E67206F6666004368617297
:105F500067696E6700506572666F726D616E63652A
:105F6000202D200052616E6765202D200053746F34
:105F700072616765202D20005374616E64617264E4
:105F8000202D2000202D204D53473A2000534D5303
:105F90002046524F4D3A20004D502D3020504100A8
:105FA0004D502D30206325642C33000D00222C3100
:105FB000350D0041542B435553443D312C22004DA7
:105FC000502D302063332C302C25642C25642C2557
:105FD00073004D502D302063312C302C25642C253E
:105FE000642C2564004D502D302061004D502D3023
:105FF00020004D502D53203020004D502D30204595
:10600000540025732C25642C25642C25642C2564D0
:106010002C25642C25642C004D502D302067002544
:10602000642C25642C25642C25642C25642C256483
:106030002C25642C256C752C25642C256C752C2541
:10604000642C25642C25642C2564004D502D3020B3
:10605000440025642E25642E25642C25732C25648C
:106060002C25642C2573004D502D302046002564CE
:1060700000302C302C0025642E25642C25642C0047
:106080004D502D302057002C25642C25642C256480
:106090002C2564004D502D30204C0025642C257596
:1060A0002C25642C25642C25642C25642C25642C3B
:1060B00025642C25642C25640025752C002C00708B
:1060C0006572666F726D616E63652C0072616E67DA
:1060D000652C0073746F726167652C007374616E58
:1060E000646172642C0073746F707065642C006856
:1060F000656174696E672C00707265706172652CE1
:1061000000646F6E652C00746F706F66662C0063A0
:1061100068617267696E672C0025642C25732C25D5
:10612000642C25642C004D502D3020530020004D50
:10613000502D43203020000D0A004D502D302045B9
:106140004D001A0041542B43495053454E440D0015
:106150004F564D53204669726D77617265207665A2
:106160007273696F6E3A2025642E25642E256400B3
:106170005045520052414E0053544F005354410079
:106180000D2025753A256400466561747572657346
:106190003A000D204E45542053746174653A3078AE
:1061A00025303278000D2047524E204C65643A2548
:1061B00064000D20524544204C65643A2564004437
:1061C0004941473A000D20506172616E6F69643A2F
:1061D0002573000D2049503A25730053657276658A
:1061E000723A000D2047534D2F475052533A204EDC
:1061F0006F7420636F6E6E656374656420283078F9
:106200002530327829000D2047534D3A204F4B0D51
:10621000205365727665723A204E6F7420636F6EFC
:106220006E6563746564000D20475052533A204FE9
:106230004B0D205365727665723A20436F6E6E6522
:1062400063746564204F4B000D2050617373776F4A
:1062500072643A2573000D20557365723A257300F8
:106260000D2041504E3A257300475052533A000DCD
:10627000204E6F74696669636174696F6E733A2545
:1062800073000D20556E6974733A2573000D205606
:10629000656869636C6549443A2573004D6F6475A0
:1062A0006C653A000D2025753A00506172616D737E
:1062B0003A002C004D6F64756C65207061737377C4
:1062C0006F72643A20257300526567697374657252
:1062D0006564206E756D6265723A20257300414CCD
:1062E00045525421212120435249544943414C20D5
:1062F000534F43204C4556454C20415050524F413E
:106300004348454420282575252520534F4329001F
:106310002575252500200D534F433A200025752073
:106320004B6D002575206D6900200D496465616C19
:106330002052616E67653A20004E6F742063686179
:106340007267696E67004368617267696E672053A0
:10635000746F70706564004368617267696E672C62
:106360002048656174696E67004368617267696E91
:10637000672C20507265706172696E6700436861B6
:106380007267696E6720446F6E650043686172676B
:10639000696E672C20546F7070696E67206F666637
:1063A000004368617267696E6700506572666F725C
:1063B0006D616E6365202D200052616E6765202D32
:1063C000200053746F72616765202D200053746143
:1063D0006E64617264202D20001A00220D0A0041B3
:1063E000542B434D47533D2200256C692E253036F2
:0363F0006C6900D5
:0C63F4006EDACED9E840E8403F0BE5D956
:106400001BDA010EAFD9EF50F00BE8380F0B006E1E
:10641000C1D9030B100DF3500010D7D9E66E010E51
:10642000A8D929DA1BE200500108000E015416E237
:10643000060E036E53DAC00B03C0E7FFE75204E019
:10644000E8427F0BE706FCE1026E010E8BD9EF50AC
:106450000F0B040DF3500210B8D901D03D0EE66EBB
:10646000020E87D908DA09E200500208000E015432
:1064700004E234DA3F0BA9D901D03D0EE66E030EDB
:1064800078D9ECD1CFD9A9D921E28DD901E3DB2A82
:10649000C0D916E1ED5014E1030EE66EE66A71D93B
:1064A000B4D901E6DFD90AE278D9EDD901E3DB2AD4
:1064B00019DADF2A010EF4E3DB2AF2D7DE6ADD6A9D
:1064C000020EDB2A030EDFE3DB2ADDD731DA0134EB
:1064D00020E200500008000E01541BE2B1D9C7D9D8
:1064E00004E6030E005C000E015804E282D9F7E3D3
:1064F000DB2AF5D702DA89D901E6B4D90AE24DD907
:10650000C2D901E3DB2AEED9DF2A010EF4E3DB2A4C
:10651000F2D7F90EDBCFE9FFFA0EDBCFEAFFEF6A25
:10652000040EE15C02E2E16AE552E16E97D17AD9AC
:1065300054D91BE238D901E3DB2A6BD910E1ED50C5
:106540000EE1030EE66EE66A1CD95FD901E68AD930
:1065500004E2CCD9FAE3DB2AF8D7DE6ADD6A020E60
:10656000DB2A030EE5E3DB2AE3D7E2D901341AE2A2
:1065700000500008000E015415E262D978D904E6F3
:10658000030E005C000E015804E233D9F7E3DB2A66
:10659000F5D7B3D93AD901E665D904E2A7D9FAE328
:1065A000DB2AF8D7040EE15C02E2E16AE552E16E13
:1065B00055D18FD9010ED6D8EF380F0B006EEAD81F
:1065C000040DF350001038D989D9E840E8403F0B5A
:1065D000006E010EC7D8EF38F00B0010E66E010E0A
:1065E000C8D8030EBFD8EFCF00F078D9400DF350D4
:1065F000C00B0010E66E020EBCD830D16AD9070E6F
:10660000E126050EDB6A060EDB6AC4D801E197D0ED
:10661000030EDB6A040EDB6A010EDB6A020EDB6A24
:106620003AD9D890015001E61DD94AE2B3D848E0E2
:10663000DF6AB0D82FE0DF502DE1FD0EDBCFE9FFA0
:10664000DB2AFE0EDBCFEAFF01E3DB2AEFCFDFFF21
:106650002B0EDF5C05E3DF507A0802E3000E01D069
:10666000010E000902E0000E09D02B0EDF5CF76A74
:10667000BB0FF66E8B0EF7220800F550DF6EDF5071
:10668000D8E0240EDF5C02E1000E02D03D0EDF5C9C
:10669000DF6ECFD77FD80CE0030EDB2A040E01E3B8
:1066A000DB2ADF5007E0DF04E66ED5D81BD902D025
:1066B000D2D8EF6A010EDB2A020EB2E3DB2AB0D792
:1066C000D950030FE96EDACFEAFFEE50ED109DE0EE
:1066D000F7D86FDFE552E552E552E552010EDB6A6D
:1066E000020EDB6AD8D8030EDBCF02F0040EDBCF3C
:1066F00003F00206000E035A01500318E8AE02D060
:10670000033404D00250005C0350015801E37DD7EC
:1067100001D9F9D8FB0EDBCFE9FFDB2AFC0EDBCF7A
:10672000EAFF01E3DB2ADED8050EDB2A060E01E3D1
:10673000DB2A010EDB2A020ED5E3DB2AD3D7B2D83F
:10674000EF6A050EDBCF00F0060EDBCF01F000C0D4
:10675000F3FF01C0F4FF070EE15C02E2E16AE552DB
:10676000E16E7CD0E76EDDD8E750E926000EEA2224
:106770001200E76E97D8E750E926000EEA2272EF82
:1067800034F09ED837DE006E060EE15E0050DE6A01
:10679000DD6A1200C6D8EF501200DECFE9FFDDCF70
:1067A000EAFF83EF34F085D8FD0EDB500024E96E5C
:1067B000FE0EDB500120EA6EEF50E66EDFCFE9FF00
:1067C000DF2A010EDBCFEAFF1200F76A7A0FF66EBE
:1067D0008B0EF7220800F55012006BD8FB0EDBCFB2
:1067E00002F0FC0EDBCF03F00250005C03500158B6
:1067F0001200020EDBCFE9FF030EDBCFEAFF9DD8CC
:10680000EF6A020EDB2A030E120092D8D8900150D4
:10681000120093D867D8D9CFE9FFDACFEAFF030E89
:10682000EE18120056D8040EE126DE6ADD6A020E6A
:10683000DB6A030EDB6A1200E66E34D872EF34F0C6
:10684000D9CFE9FFDACFEAFF020EEECFDBFF030E6E
:10685000EDCFDBFF12005ED89DEF34F0E552E7CFBD
:10686000D9FF1200040E005C000E0158120021D85E
:10687000D89001501200F90EDBCF00F0FA0EDBCFFA
:1068800001F001341200F90EDBCFE9FFDB2AFA0E2A
:10689000DBCFEAFF1200010EDBCF00F0020EDBCFF0
:1068A00001F01200FB0EDBCFE9FFFC0EDBCFEAFFAD
:1068B0001200020EDBCF00F0030EDBCF01F012005E
:1068C000F30EE66E080EE66EEF0EE66E080EE66E4E
:1068D0001200D9CFE6FFE1CFD9FF1200020E42DF4E
:1068E000EF501200E552E750EF6E120056DF17EC42
:1068F0001AF0E552DF2A010E1200DECFE6FFDDCFEF
:10690000E6FFC1EF33F0F30EE926080EEA22EF505E
:10691000E66E1200010EDBCFE9FF020EDBCFEAFFCD
:106920001200FD0EDBCFE9FFFE0EDBCFEAFF120007
:10693000DECF00F0DDCF01F01200EF0EE926080EE9
:04694000EA22120035
:0C694400219E05D0219E29AE02D0296CB6
:10695000218E29C023F0226A336A326A860E246EA1
:10696000256A88EF36F0219E08D0219E29AE05D0F9
:10697000286C291EE86A2922218E29C023F028C00C
:1069800022F0336A326A8E0E246E256A88EF36F062
:10699000219E0CD0219E29AE09D0266C271E281ED0
:1069A000291EE86A272228222922218E29C023F0C5
:1069B00028C022F027C033F026C032F09E0E246E8D
:1069C000256A88EF36F0216AC4EC36F0DCEC36F04C
:1069D00021B66CEF36F021A205D021BA6CEF36F06B
:1069E00073EF36F021BA7FEF36F021A005D021B841
:1069F0006CEF36F07FEF36F021B873EF36F0256A92
:106A00007F0E2A24246EE86A25222F50245EE86A2D
:106A1000255A1A0E306E2A6A326A336A226A236A4B
:106A20002C50275E2D50285A2E50295A000E2A5AD3
:106A300009E72C5027262D5028222E502922000EFF
:106A40002A2201D0328AD8902736283629362A368B
:106A5000D8903236333622362336302EE1D72950BD
:106A600028102710D8A4328A88EF36F0216AC4ECA7
:106A700036F0DCEC36F021B66CEF36F021A205D012
:106A800021B86CEF36F073EF36F021AA05D021B0B3
:106A90006CEF36F073EF36F021B002D021A802D0AF
:106AA0007FEF36F0256A2F502A24246EE86A2522CB
:106AB0007E0E245EE86A255A326A336A226A236AA5
:106AC0002E502902F4CF23F0F3CF22F02D502902CB
:106AD000F3503326F4502222000E23222E50280297
:106AE000F3503326F4502222000E23222C50290288
:106AF000F3503226F4503322000E222223222D504E
:106B00002802F3503226F4503322000E2222232290
:106B10002E502702F3503226F4503322000E222248
:106B200023222C502802F4503226000E3322222237
:106B300023222D502702F4503226000E3322222227
:106B4000232288EF36F0206A2EAEA9EF35F02E6CA6
:106B5000201E29AEAEEF35F0296C201E29EC47F03F
:106B600029BEB8EF35F020AE000C296C256C000C66
:106B700020BEB5EF35F02188FF0C206A2EAEC6EF9F
:106B800035F02D6C2E1EE86A2E22201E29AECEEF87
:106B900035F0286C291EE86A2922201ED5EC46F023
:106BA00029BEDEEF35F020AE000C286C291EE86A05
:106BB0002922246C251EE86A2522000C20BED5EF70
:106BC00035F02188FF0C206AE86A2EAEF0EF35F030
:106BD0002B6C2C1E2D1E2E1E2C222D222E22201E12
:106BE00029AEFBEF35F0266C271E281E291E272212
:106BF00028222922201EB1EC46F029BE12EF36F0E1
:106C000020AE000C266C271E281E291EE86A2722AB
:106C100028222922226C231E241E251E2322242200
:106C20002522000C20BE02EF36F02188FF0C28C080
:106C300032F028502D02F4CF27F0F3CF26F0295060
:106C40002E02F4CF29F0F3CF28F02D02F35027269F
:106C5000F4502822E86A292232502E02F3502726C7
:106C6000F4502822E86A2922000C216AC4EC36F08C
:106C700021B63FEF36F021A20FD021B407D07F0E0E
:106C8000296EFF0E286E276E266E25D0800E296E87
:106C900001D0296A000EF6D721B0FBD7266A9F0ED5
:106CA0002A60EBD77E0E2A64F4D79E0E2A5C07E09A
:106CB000D89029322832273226322A2AF6D721A420
:106CC0000AD0266C271E281E291EE86A27222822A1
:106CD000292229AEDED712007F0E2A6EFF0E296E02
:106CE000286E276E12007F0E21BEFF0E2A6E02D084
:106CF0007F0E2A6E800E296E286A276AF3D721AE8E
:106D000004D0800E2A6E296AF7D72A6A296AF4D736
:106D10002350221033103210F8E025BEF0D723BEE6
:106D20000CD024502510EBE0D89032363336223682
:106D300023362406D8A02506F2D72550D4E12428EE
:106D4000D2E032AE11D07F0E321402E133A00CD06B
:106D5000332AE86A2222232207E3D8802332223210
:106D60003332242A2428BFE02450C9E033C027F05E
:106D700022C028F02334296E24302A6E29322A9E1C
:106D800021BE2A8E72EF36F029362A3602E321849C
:106D9000217E06E121802A6A296A286A276A120070
:106DA0002A2803E0D88029321200D890293202E143
:106DB00021821200218612002E362F3602E3218C0A
:106DC000217E06E121882F6A2E6A2D6A2C6A120024
:106DD0002F2803E0D8802E321200D8902E32EAE11C
:106DE000218A120029C033F028C032F028502D0229
:106DF000F4CF27F0F3CF26F029502E02F4CF29F05C
:106E0000F3CF28F02D02F3502726F4502822E86A09
:106E1000292232502E02F3502726F4502822E86A05
:106E200029222EAE18EF37F03250285E3350295AFF
:0E6E300033AE000C2D50285E2E50295A000C57
:026E3E0050659D
:106E4000726D697373696F6E2064656E6965640045
:106E5000596F75722070686F6E652068617320626B
:106E600065656E207265676973746572656420611B
:106E70007320746865206F776E65722E004D6F64A5
:106E8000756C652070617373776F726420686173CD
:106E9000206265656E206368616E6765642E0050D0
:106EA0006172616D657465727320686176652062D8
:106EB00065656E207365742E004665617475726534
:106EC00020686173206265656E207365742E0048CA
:106ED0006F6D656C696E6B20616374697661746552
:106EE000640056656869636C65206C6F636B207223
:106EF00065717565737465640056656869636C6572
:106F000020756E6C6F636B20726571756573746547
:106F1000640056616C6574206D6F646520726571E4
:106F20007565737465640056616C6574206D6F647B
:106F3000652063616E63656C20726571756573743D
:106F4000656400436861726765206D6F64652063E6
:106F500068616E676520726571756573746564003C
:106F60004368617267652073746172742072657121
:106F70007565737465640043686172676520737436
:106F80006F702072657175657374656400547275F5
:106F90006E6B20686173206265656E206F70656E30
:106FA0006564202876616C6574206D6F6465292E98
:106FB00000436172206C6F636174696F6E3A0D6893
:106FC0007474703A2F2F6D6170732E676F6F676CDA
:106FD000652E636F6D2F6D6170732F6170692F73F4
:106FE00074617469636D61703F7A6F6F6D3D3135A7
:106FF0002673697A653D35303078363430267363D0
:10700000616C653D322673656E736F723D66616CAF
:107010007365266D61726B6572733D69636F6E3A5D
:10702000687474703A2F2F676F6F2E676C2F7042E1
:107030006358372537430052454749535445523F1B
:107040000000000000000000000000000000000040
:1070500000005245474953544552000000000000CB
:10706000000000000000000000000000005041533C
:10707000533F00000000000000000000000000007E
:1070800000000000000000005041535320000000A9
:1070900000000000000000000000000000000000F0
:1070A00000000047505300000000000000000000F6
:1070B0000000000000000000000000000000535429
:1070C000415400000000000000000000000000002B
:1070D000000000000000000000504152414D533FAD
:1070E00000000000000000000000000000000000A0
:1070F00000000000504152414D53200000000000AC
:107100000000000000000000000000000000004D32
:107110004F44554C453F00000000000000000000B7
:10712000000000000000000000004D4F44554C4599
:10713000200000000000000000000000000000002F
:107140000000000000475052533F000000000000C4
:10715000000000000000000000000000000000002F
:1071600047505253200000000000000000000000C3
:10717000000000000000000000000053455256458A
:10718000523F00000000000000000000000000006E
:1071900000000000000053455256455220000000F8
:1071A00000000000000000000000000000000000DF
:1071B00000444941470000000000000000000000BA
:1071C000000000000000000000000000464541549F
:1071D000555245533F000000000000000000000031
:1071E0000000000000000046454154555245200073
:1071F000000000000000000000000000000000008F
:107200000000484F4D454C494E4B20000000000007
:10721000000000000000000000000000004C4F4390
:107220004B200000000000000000000000000000F3
:107230000000000000000000554E4C4F434B200062
:10724000000000000000000000000000000000003E
:1072500000000056414C4554200000000000000092
:107260000000000000000000000000000000554E7B
:1072700056414C4554200000000000000000000072
:107280000000000000000000004348415247454D07
:107290004F444520000000000000000000000000F6
:1072A00000000000434841524745535441525400A6
:1072B000000000000000000000000000000000438B
:1072C000484152474553544F500000000000000011
:1072D0000000000000000000000056455253494FD6
:1072E0004E00000000000000000000000000000050
:1072F000000000000052455345540000000000000B
:10730000000000000000000000000000000000007D
:10731000000000000000000000000000000000006D
:0B732000000000000000000000000062
:04732C00FB0EE3CFA2
:10733000F6FFFC0EE3CFF7FFFD0EE3CFF8FFFE0EE6
:10734000E3CFE9FFFF0EE3CFEAFFF90EE35003E1DD
:10735000FA0EE35009E0F90EE30602E2FA0EE30644
:107360000900F550EE5CF1E01200D9CFE6FFDACF6C
:10737000E6FFFA0EE3CFD9FFFB0EE3CFDAFFFC0EF8
:10738000E3CFE9FFFD0EE3CFEAFFE9CFF3FFEACF5A
:10739000F4FFF80EE35003E1F90EE35008E0F80EB5
:1073A000E30602E2F90EE306DECFEEFFF2D7FF0EB0
:1073B000E3CFDAFFE552FF0EE3CFD9FFE55212002B
:1073C000FE0EE3CFE9FFFF0EE3CFEAFFE9CFF3FFC5
:1073D000EACFF4FFFB0EE35003E1FC0EE35009E0BB
:1073E000FB0EE30602E2FC0EE306FD0EE350EE6E3A
:1073F000F1D71200D9CFE6FFDACFE6FFFA0EE3CFDE
:10740000D9FFFB0EE3CFDAFFFC0EE3CFE9FFFD0E61
:10741000E3CFEAFFE9CFF3FFEACFF4FFEE66FED752
:10742000ED52DFCFEEFFDE66FCD7FF0EE3CFDAFFD3
:10743000E552FF0EE3CFD9FFE5521200FB0EE3CF7A
:10744000F6FFFC0EE3CFF7FFFD0EE3CFF8FFFE0ED5
:10745000E3CFE9FFFF0EE3CFEAFFE9CFF3FFEACF87
:10746000F4FFEE66FED7ED520900F5CFEFFFEE66B2
:10747000FBD71200D9CFE6FFDACFE6FFFA0EE3CF53
:10748000D9FFFB0EE3CFDAFFFC0EE3CFE9FFFD0EE1
:10749000E3CFEAFFDE50EF5C02E1EE66FBD7F36E6E
:1074A000FF0EE3CFDAFFE552FF0EE3CFD9FFE5523F
:1074B000F3501200D9CFE6FFDACFE6FFFA0EE3CFA2
:1074C000D9FFFB0EE3CFDAFFFC0EE3CFE9FFFD0EA1
:1074D000E3CFEAFFE9CFF3FFEACFF4FFDECFEFFF20
:1074E000EE66FCD7FF0EE3CFDAFFE552FF0EE3CFE7
:1074F000D9FFE5521200FB0EE3CFF6FFFC0EE3CFFF
:10750000F7FFFD0EE3CFF8FFFE0EE3CFE9FFFF0E1E
:10751000E3CFEAFFE9CFF3FFEACFF4FF0900F5CFAD
:10752000EFFFEE66FBD71200FE0EE3CFE9FFFF0E82
:10753000E3CFEAFFF36AF46AEE5203E0F34AF42A77
:10754000FBD71200FF0EE3CFF8FFE552FF0EE3CFAB
:10755000F7FFE552FF0EE3CFF6FFE552E66AE66A73
:10756000E66A0900F55209E0FD0EE32A05E1FE0E88
:10757000E32A02E1FF0EE32AF4D7FD0EE3CF27F062
:10758000FE0EE3CF28F0FF0EE3CF29F01200D9CF93
:10759000E6FFDACFE6FFFA0EE3CFD9FFFB0EE3CF2B
:1075A000DAFFFC0EE3CFE9FFFD0EE3CFEAFFF80EB2
:1075B000E35003E1F90EE3500AE0F80EE30602E2BD
:1075C000F90EE306DE50EF5C02E1EE66F0D7F36EF3
:1075D000FF0EE3CFDAFFE552FF0EE3CFD9FFE5520E
:1075E000F3501200D9CFE6FFDACFE6FFFA0EE3CF71
:1075F000D9FFFB0EE3CFDAFFFC0EE3CFE9FFFD0E70
:10760000E3CFEAFFE9CFF3FFEACFF4FFF80EE35050
:1076100003E1F90EE3500BE0F80EE30602E2F90E87
:10762000E306DECFEFFFEE66F1D7DD52EFD7FF0EB8
:10763000E3CFDAFFE552FF0EE3CFD9FFE5521200A8
:10764000FE0EE3CFF3FFFF0EE3CFF4FFFB0EE3CF1D
:10765000F6FFFC0EE3CFF7FFFD0EE3CFF8FFF3CF0D
:10766000E9FFF4CFEAFF0900F5500CE0F550EF5CBC
:1076700002E1EE52F8D7EF5203E0F34AF42AE6D7DC
:10768000F36AF46A1200FE0EE3CFE9FFFF0EE3CFC8
:10769000EAFFE9CFF3FFEACFF4FF610EEF5C05E606
:1076A0007B0EEF5C02E7DF0EEF16EE52F6E1120002
:1076B000DACFE4FFE2CFDAFFE9CFE4FFEACFE4FF7D
:1076C000F6CFE4FFF7CFE4FFF5CFE4FFF3CFE4FF1D
:1076D000F4CFE4FFFACFE4FF00EE20F0140EE8044C
:1076E00003E3EECFE4FFFBD700EE00F0200EE8044A
:1076F00003E3EECFE4FFFBD7E65260BE76D80F017E
:1077000050BF89D8A46AE55200EE1FF0200EE804AD
:1077100003E3E5CFEDFFFBD700EE33F0140EE804F2
:1077200003E3E5CFEDFFFBD7E5CFFAFFE5CFF4FFAD
:10773000E5CFF3FFE5CFF5FFE5CFF7FFE5CFF6FFA8
:10774000E5CFEAFFE5CFE9FFE5CFDAFF11003AD94F
:107750000801560EC76F410EC86FC96B900E6F6E51
:107760006EAEFED7606A0F01A00E196F1869016B2B
:10777000200E006F506BE00E1D6F1C69800E096FAC
:10778000680E086F400E0D6F800E0C6F116B106F3E
:10779000706AD20E716E020E726E200E736E080148
:1077A000DB51000802E26F6A02D0600E6F6ED08E6D
:1077B000A382A380030EA56E020EE66EA3EC3FF03B
:1077C000E552F3CFDEFFF4CFDDFFDECFE9FFDDCF03
:1077D000EAFFEFCFFEF70801E56BED6B020EE15C0F
:1077E00002E2E16AE552E16EF9D00F0E651408017C
:1077F000DC6F66CFDDF867CFDEF868CFDFF869CFE2
:10780000E0F86ACFE1F86BCFE2F86CCFE3F86DCF28
:10781000E4F8609E1200D9CFE6FFE1CFD9FFE6522F
:107820000F0E0F0155150801DC6F56CFDDF857CF4D
:10783000DEF858CFDFF859CFE0F85ACFE1F85BCF48
:10784000E2F85CCFE3F85DCFE4F850CFDFFF0F0143
:10785000509FE552C3D0000E0901E76E5419E8AEFF
:1078600002D0543503D0E750D880545501E2540774
:10787000000E0901E76E5519E8AE02D0553503D068
:10788000E750D880555501E25507000E0901E76E13
:107890005619E8AE02D0563503D0E750D880565579
:1078A00001E25607000E0901E76E5719E8AE02D053
:1078B000573503D0E750D880575501E257071200DB
:1078C00081D80801D551DE6EDD6A0701FB5117E151
:1078D00070D801500318E8AE02D0033404D002502F
:1078E000005C035001580BE2020EE66EE66A24ECDF
:1078F0001AF0E552E5520701010EFB6F15D00701A2
:10790000FB0512E156D8020E0226000E0322035098
:107910000118E8AE02D0013404D00050025C0150DE
:10792000035802E20701FB6B020EE15C02E2E16A2E
:10793000E552E16E53D0120012000701FC2B000E3D
:10794000FD2389DF46D83C0E2D6E2E6A22D801E138
:10795000B7DF3FD82C0E2D6E010E2E6E1AD801E126
:10796000EADF37D8580E2D6E020E2E6E12D806E1C1
:10797000E3DF580E0701FC5F020EFD5B12001200F0
:1079800012001200120012D011D010D00FD00ED061
:107990000DD0FCC728F0FDC729F0D5EC46F024C077
:1079A00000F025C001F0245025101200D9CFE6FFC9
:1079B00015D009011351006E016ADECF02F0DDCF50
:1079C00003F01200D9CFE6FFE1CFD9FF020EE12686
:1079D0001200FCC700F0FDC701F01200E552E7CF2E
:0479E000D9FF1200B9
:0C79E400D9CFE6FFE1CFD9FF0A0EE12663
:1079F000020EDB6A030EDB6A040EDB6A050EDB6A2D
:107A00001CD9EF6A1AD9EE52EF6A2FD9080EE9CFC6
:107A1000DBFF090EEACFDBFFDE6ADD6A2DD904E663
:107A2000000E005C010E015808E201D9DFCFEFFF24
:107A3000DF2A010EF3E3DB2AF1D7DE6ADD6A1CD907
:107A400004E6000E005C010E01586BE2F0D8EF5026
:107A5000E66ED950060F01D9060EDBCF02F0070EF5
:107A6000DBCF03F0020EDB500224006E030EDB506E
:107A70000320040EDBCF06F0050EDBCF07F0F90E76
:107A8000DB500624E96EFA0EDB500720EA6EEF5059
:107A9000046E056A00500424E66ED950020FDDD84A
:107AA000020EDBCF02F0030EDBCF03F0080EDB503B
:107AB0000224E96E090EDB500320EA6EEF50E66EF9
:107AC000B6D8E552E750EF6E020EDBCF00F0030EA2
:107AD000DBCF01F0080EDB500024E96E090EDB500D
:107AE0000120EA6E060EDBCFEFFF040EDB2ADBCFB0
:107AF00000F0050E01E3DB2ADBCF01F0A5D8E8AEEC
:107B000002D0033404D00250005C0350015804E357
:107B1000040EDB6A050EDB6ADF2A010E90E3DB2A26
:107B20008ED70A0EE15C02E2E16AE552E16EE552AF
:107B3000E7CFD9FF1200D9CFE6FFE1CFD9FF080E7A
:107B4000E1267BD8040EEFCFDBFF77D8EE52050E8F
:107B5000EFCFDBFF8AD8020EE9CFDBFF030EEACFBF
:107B6000DBFFDE6ADD6ADECF00F0DDCF01F06CD82E
:107B7000E8AE02D0033404D00250005C0350015838
:107B800037E2040EDB2ADB5046D8060EEFCFDBFFD0
:107B9000050EDBCFE7FF060EDB50E726050EE7CF2D
:107BA000DBFFDB5038D8070EEFCFDBFF040EDB50D6
:107BB00032D8070EDBCFEFFF050EDB502CD8060EB8
:107BC000DBCFEFFF070EDBCFE6FF060EDB50E55203
:107BD000E72421D8EFCF02F0F90EDBCF00F0FA0E48
:107BE00052D80250EF1ADF2A010EBDE3DB2ABBD7C1
:107BF00024D8040EDBCFEFFF20D8EE52050EDBCFEA
:107C0000EFFF080EE15C02E2E16AE552E16EE55247
:107C1000E7CFD9FF1200E76E020EDBCFE9FF030EBC
:107C2000DBCFEAFFE750E926000EEA221200080E39
:107C3000DBCF00F0090E43EF3EF0FD0EDBCFE9FF96
:107C4000FE0EDBCFEAFF1200F70EDBCF02F0F80EDC
:107C5000DBCF03F0015003181200E96EDACFEAFF20
:107C6000E552E750EE6EED6A1200FB0EDBCFE9FF46
:107C7000FC0EDBCFEAFF1200DECF00F0DDCF01F01B
:107C8000D89001501200DBCF01F0DE500024E96EE5
:087C9000DD500120EA6E120034
:087C9800FF0012004ED9E65274
:107CA000DF6A7C0ECA6ECC6ACB687A0EDF5C05E2B6
:107CB0009EA2FED79E92DF2AF8D7E55231D13DD958
:107CC000FE0EDB50000804E2E9DFFE0EDB06F8D70B
:107CD00027D1D9CFE6FF24D1D9CFE6FF21D181B07A
:107CE00005D08180050EE66EEADFE5528190140E24
:107CF000E66EE5DFE552818012001FD90C0EE12609
:107D0000D950FB0FE96EFF0EDA20EA6ED890030E11
:107D1000EB50000A08E6000EEE5C000EEE58000E76
:107D2000EE58000EEE5827E2F90EDBCFE9FFDB2A12
:107D3000FA0EDBCFEAFF01E3DB2A2D0EEF6EFB0E1E
:107D4000DBCF00F0FC0EDBCF01F0FD0EDBCF02F04D
:107D5000FE0EDBCF03F0001E011E021E031EFB0EF3
:107D600000C0DBFFFC0E01C0DBFFFD0E02C0DBFF2D
:107D7000FE0E03C0DBFFFB0EDBCF08F0FC0EDBCFFB
:107D800009F0FD0EDBCF0AF0FE0EDBCF0BF0CCD8F6
:107D9000CAEC34F027C004F028C005F029C006F072
:107DA0002AC007F02C6A2D6A2E6A450E2F6EE3EC6E
:107DB00034F027C000F028C001F029C002F02AC02A
:107DC00003F02C6A2D6A610E2E6E450E2F6EE3ECC9
:107DD00034F027C0DEFF28C0DEFF29C0DEFF2AC046
:107DE000DDFFDD52DD52DECF27F0DECF28F0DECF23
:107DF00029F0DDCF2AF0DD52DD5235EC36F0040EED
:107E000026C0DBFF050E27C0DBFF060E28C0DBFF08
:107E1000070E29C0DBFF040EDBCF08F0050EDBCF19
:107E200009F0060EDBCF0AF0070EDBCF0BF0400E99
:107E30002B6E420E2C6E0F0E2D6E2E6A75D848ECEE
:107E400046F022C008F023C009F024C00AF025C083
:107E50000BF0D9CFE9FFDACFEAFFEECF04F0EECF97
:107E600005F0EECF06F0EFCF07F02C6A240E2D6E52
:107E7000740E2E6E490E2F6E04C027F005C028F038
:107E800006C029F007C02AF036EC35F035EC36F0A4
:107E900000010850265C006E09502758016E0A50F8
:107EA0002858026E0B502958036E080E00C0DBFFE5
:107EB000090E01C0DBFF0A0E02C0DBFF0B0E03C080
:107EC000DBFFD950080F20D8D950040F1DD8E90E78
:107ED000006E630E016E026A00C0E6FFE66E02C02D
:107EE000E6FFF90EDBCFE6FFFA0EDBCFE6FFC9ECCB
:107EF00044F0036E0D0EE15E03500C0EE15C02E2F5
:107F0000E16AE552E16E0CD0E96EDACFEAFFEECF1E
:107F1000E6FFEECFE6FFEECFE6FFEFCFE6FF120083
:107F2000E552E7CFD9FF120008C026F009C027F0BC
:107F30000AC028F00BC029F01200D9CFE6FFE1CF2C
:047F4000D9FF120053
:0C7F44001200D9CFE6FFE1CFD9FF040EF8
:107F5000E126A66AFE0EDB50E66ED950020FB0D8BD
:107F6000020EDBCF2DF0030EDBCF2EF017EC36F038
:107F7000020E26C0DBFF030E27C0DBFF020E030E3E
:107F8000AAD8020EDBCF00F0030EAFD8C1D804E6AA
:107F9000200E005C000E01580AE2A680B0D8A8CFDF
:107FA000EFFFA92ADF2A010EF1E3DB2AEFD7DD0E6E
:107FB000006E090E016E00C0F3FFF46E040EE15C6A
:107FC00002E2E16AE552E16EE552E7CFD9FF120025
:107FD000D9CFE6FFE1CFD9FF050EE126DE6ADD6AE3
:107FE000200EE66EE66AFC0EDBCFE6FFFD0EDBCF71
:107FF000E6FFDD0EE66E090EE66EF2EC3AF0006E7C
:10800000060EE15E00500901FC6BFE0EDB50E66ED1
:10801000D950030F55D8030EDBCF2DF0040EDBCF64
:108020002EF017EC36F0030E26C0DBFF040E27C03F
:10803000DBFF030EDBCF00F0040E4DD8030EDBCFC9
:1080400000F0040E52D864D804E6200E005C000E46
:1080500001582CE2FE0EDB50200DF3CF02F0F4CFDE
:1080600003F0000E0226000E0322DE500224006EF2
:10807000DD500320016E0050A96EA66AA6843FD889
:10808000EF50A86E020EF2CFDBFFF29E550EA76EE8
:10809000AA0EA76EA682020EDB50F26EA6B2FED723
:1080A000A694DF2A010ECFE3DB2ACDD7050EE15CD3
:1080B00002E2E16AE552E16EE552E7CFD9FF120034
:1080C000E96EDACFEAFFE552E750EE6EED6A200E78
:1080D000286E296A1200DBCF01F001C000F0016AAE
:1080E0000050AA6EFF0EE76E1200DBCF01F0E750E2
:1080F0000016016A0050A96EDE6ADD6A1200DECF4A
:10810000E9FFDDCFEAFFDD0EE926090EEA221200C3
:0E811000DECF00F0DDCF01F0D890015012005C
:02811E00D9CFB7
:10812000E6FFE1CFD9FF040EE126DF6A080EDF5C2F
:1081300009E2DF50EA6ACC0FE96E080EEA22EF6A24
:10814000DF2AF4D7080EDF6E100EDF5C20E2080E87
:10815000DF5C180FE66EA3EC3FF0E552F3CF00F0C2
:10816000F4CF01F000C0E6FF01C0E6FFCFEC43F022
:10817000E552E552F350E66EDF50EA6ACC0FE96E45
:10818000080EEA22E552E750EF6EDF2ADDD780ECD9
:1081900046F0FE0E936E870ED56E3BEC43F0A2ECDC
:1081A0003FF0A7EC3BF0F6EC1FF00A0EE66E5FEC3A
:1081B0003EF0E552E668E66A11EC43F0E552E5521E
:1081C000E66A010EE66E11EC43F0E552E55238EC3A
:1081D00043F00A0EE66E5FEC3EF0E55200C9E6FFA2
:1081E000010EE66E11EC43F0E552E55238EC43F037
:1081F000230EE66E5FEC3EF0E552040001C9E6FF97
:10820000010EE66E11EC43F0E552E55238EC43F016
:10821000230EE66E5FEC3EF0E552040002C9E6FF75
:10822000010EE66E11EC43F0E552E55238EC43F0F6
:10823000230EE66E5FEC3EF0E5520400E66A010EA6
:10824000E66E11EC43F0E552E552E66AE66A11EC9F
:1082500043F0E552E55238EC43F00A0EE66E5FEC6F
:108260003EF0E55204000A0EE66E010EE66E11ECD9
:1082700043F0E552E55238EC43F0010EDB6A0801A9
:1082800008010051200B05E1080108010051100B05
:1082900002E012EC19F0080100B702D015EC19F059
:1082A000C0EC3CF00400D650DF6E4C0ED75C07E308
:1082B000D76AD66ABCEC1FF09DEC3CF00ED0010EE4
:1082C000DB50D75C0AE0D750030B04E1F5EC1FF05C
:1082D000BFEC3CF0010ED7CFDBFFD1D7040EE15C41
:1082E00002E2E16AE552E16EE552E7CFD9FF120002
:1082F000080100910083416B426B436B009500873E
:10830000009B0099C46BC56BC66B810EAF6EAC84CD
:10831000949C948E9F989F9AAC8AAB88AB8E9D88D4
:108320009D8AF28EF28C1200AFD8080100A102D013
:10833000000E17D09D984251EA6A010FE96E080EAF
:10834000EA22FE0EDBCFEFFF0093412B400E415D92
:1083500001E10081422B400E425D01E1426B9D88AC
:10836000010E97D0400E0801415D04E2400ED88016
:1083700041551200000C88D8080100A702D0000E59
:1083800020D09D9A0095C651EA6A440FE96E080E06
:10839000EA22EF50E66EFD0EDBCFE9FFFE0EDBCFEB
:1083A000EAFFE552E750EF6EC407C45101E10087D0
:1083B000C62BC65172D803E1015001E1C66B9D8AFC
:1083C000010E67D00801C45112005ED8E6529D50DC
:1083D000100B01E0010E006E9E50100B01E0010E2B
:1083E000001419E0080100B314D04351EA6A010FE8
:1083F000E96E080EEA22EF50AD6E00B10091410720
:10840000415101E10083432B400E435D3BE1436B4F
:1084100039D09D9837D09D50200B01E0010E006EA1
:108420009E50200B01E0010E00142CE0ABB404D0F0
:10843000ABA207D0AB98AB88AE50DF6E0801008BC3
:1084400021D0080100A504D0AE50DF6E00891AD0FB
:1084500000B518D000990097C551EA6A440FE96E3B
:10846000080EEA22AECFEFFFC42BC45116D803E1A9
:10847000015001E10085C52BC5510FD803E1015022
:1084800001E1C56BE55205D0D9CFE6FFE1CFD9FFB9
:108490001200E552E7CFD9FF1200006E016A800E8C
:0484A00000181200AE
:0C84A400D9CFE6FFE1CFD9FF020EE126A0
:1084B000400EE66EE66AE66A000EE66E040EE66EB2
:1084C000E0EC39F0006E050EE15E0050400EE66E05
:1084D000E66AE66A400EE66E040EE66EE0EC39F0FF
:1084E000006E050E76D8000EE66E040EE66EB5EC54
:1084F00039F0006E060E6DD8400EE66E040EE66E84
:10850000B5EC39F0006E060EE15E0050DE6ADD6A01
:10851000DECF00F0DDCF01F0D890015004E6400E30
:10852000005C000E01581DE2360E006EDECFE9FF42
:10853000DDCFEAFF000EE926040EEA220050EF1A12
:108540005C0E006EDECFE9FFDDCFEAFF400EE926CC
:10855000040EEA220050EF1ADF2A010ED9E3DB2ACB
:10856000D7D746D8000EE66E040E4BD8FB0EDBCFF5
:10857000E6FFFC0EDBCFE6FFFD0EDBCFE6FFFE0ED7
:1085800017D836D8400EE66E040E3BD8100EE66EB5
:10859000E66AF50EDBCFE6FFF60E0AD8020EE15CC6
:1085A00002E2E16AE552E16EE552E7CFD9FF12003F
:1085B000DBCFE6FF29D830D8F50EDBCFE6FFF60E8D
:1085C000DBCFE6FFB0EC01F0E552E552E552E552B3
:1085D0001200E15E0050F70EDBCFE6FFF80EDBCFB6
:1085E000E6FFF90EDBCFE6FFFA0EDBCFE6FF120067
:1085F00013D840EC00F0E552E552400EE66EE66A14
:108600001200E66E04EF43F007D883EC00F0006E32
:10861000060EE15E00501200800EE66E040EE66E5D
:02862000120046
:0E862200D9CFE6FFE1CFD9FFFE0EDB50EA6AAA
:10863000FB0FE96E060EEA22FD0EDBCFEFFFDB50EB
:10864000FF0812E1FD0EDB50040F006E010E005218
:1086500002E0A1D8FEE18212FE0EDB50EA6AFD0FB5
:10866000E96E060EEA22EF6AE552E7CFD9FF120063
:108670000601FF6B1200CF0E8216B50ECD6E9F90D5
:108680009D80CE6ACF6A12009EA06FD00601FF3592
:1086900002E3FF2B69D0FF5127E10701FF6B020EB8
:1086A000FF5D1FE270D8E66E61D8E552E750EF6ECD
:1086B0006AD805E162D810E06ED8FEE10DD063D82B
:1086C000FF0806E15AD802E066D8FEE1821206D021
:1086D00054D802E060D8FEE1E81C82160701FF2BA7
:1086E000DED706011F0E03D0FF0503E1F60EFF6F74
:1086F0003BD0FF070701FF6B020EFF5D35E236D866
:10870000EFCF00F0000EE76E0018E8AE02D00034A4
:1087100003D0E750D88000541BE2FFC629F0030EB7
:108720002E6EA3EC35F0255009E107011FD8EF06A6
:1087300024D802E030D8FEE1821213D0040E0701E3
:10874000FF25006E010E00520AE025D8FEE107D099
:108750000DD8EF5006E111D802E01DD8FEE1E81C6B
:1087600082160701FF2BC8D79E901200FF51EA6ABC
:10877000FD0FE96E060EEA221200040EFF25006EC0
:10878000010E00521200FF51EA6AFB0FE96E060E5D
:0E879000EA22EF501200E846FE0B000612002F
:02879E00FF0ECC
:1087A000E3CFEAFFE552FF0EE3CFE9FFE552E66AC9
:1087B000E66AD9CFE6FFDACFE6FFFC0EE124D96EF8
:1087C000FF0EE220DA6EE66AE66AE66A200EEF5CE9
:1087D00006E0090EEF5C03E0EF6603D03FD0EE50F9
:1087E000F5D72D0EEF5C03E1FF0EE32A03D02B0E2D
:1087F000EF5C01E1EE502F0EEF6424D03A0EEF60F3
:1088000021D0D890F90EE336FA0EE336FD0EDECF16
:10881000E3FFFE0EDDCFE3FFD890F90EE336FA0E4C
:10882000E336D890F90EE336FA0EE336FD0EE35048
:10883000DE26FE0EE350DD22300EEE5CDE26000E5C
:10884000DD22D9D7FF0EE3CFE8FFE85207E0F90EAB
:10885000E31EE32AFA0ED8B4E306E31EE552E5521E
:10886000E552FF0EE3CFDAFFE552FF0EE3CFD9FF6B
:10887000E552E1CFE9FFE2CFEAFFED52ED52EECF54
:10888000F3FFEFCFF4FF1200FE0EE3CFFEF4FF0E76
:10889000E3CFFFF41200FFC429F0FEC428F0350E28
:1088A0002D6E450E2E6E17EC36F0262AE86A27222A
:1088B000279E27C0FFF426C0FEF4FEC4F3FFFFC4CA
:0488C000F4FF1200AF
:0C88C4004D502D30206325642C30004DF9
:1088D000502D30206325642C312C496E76616C69F3
:1088E000642073796E746178004D502D30206325BB
:1088F000642C312C4E6F207772697465206163633C
:1089000065737320746F2043414E004D502D30200D
:108910006325642C312C506172616D657465722021
:108920006F7574206F662072616E6765004D502D03
:1089300030206325642C312C43616E6E6F7420638C
:108940006861726765202863686172676520706F6F
:10895000727420636C6F73656429004D502D302054
:108960006325642C312C43616E6E6F742073746FB9
:10897000702063686172676520286368617267654B
:10898000206E6F7420696E2070726F6772657373EA
:028990002900BC
:0E899200D9CFE6FFDACFE6FFE1CFD9FFE2CF83
:1089A000DAFFE652E652E652E652D950F90F006E6F
:1089B000FF0EDA20016E020E00C0DBFF030E01C0C5
:1089C000DBFF020EDBCFE6FF030EDBCFE6FFF90E87
:1089D000DBCFE6FFFA0EDBCFE6FFFB0EDBCFE6FFD9
:1089E000D950FC0FE66EFF0EDA20E66EB7EC28F0E9
:1089F000006E070EE15C02E2E16AE552E16E0050B2
:108A0000F3CFDEFFF4CFDDFFFC0EDBCFE9FFFD0E81
:108A1000DBCFEAFFEF6ADECF00F0DDCF01F000C070
:108A2000F3FF01C0F4FF040EE15C02E2E16AE552EB
:0E8A3000E16EE552E5CFDAFFE7CFD9FF120085
:028A3E001E0E0A
:108A4000F66E000EF76E000EF86E07010900F55085
:108A5000F66F0900F550F76F03E1F66701D03DD0DE
:108A60000900F550F16F0900F550F26F0900F5505B
:108A7000F36F09000900F550E96E0900F550EA6E40
:108A8000090009000900F550F46F0900F550F56F71
:108A900009000900F6CFF8F7F7CFF9F7F8CFFAF7A2
:108AA000F1C7F6FFF2C7F7FFF3C7F8FF0701F4536A
:108AB00002E1F55307E00900F550EE6EF407F8E225
:108AC000F507F9D7F8C7F6FFF9C7F7FFFAC7F8FFB8
:0C8AD0000701F607000EF75BBFD712008D
:048ADC0041542B4393
:108AE000534D494E533F0D0041542B4350494E3F87
:108AF0000D0041542B4950523F3B2B435245473DBB
:108B0000313B2B434C49503D313B2B434D47463D78
:108B1000313B2B434E4D493D322C323B2B4353448A
:108B2000483D313B2B434950535052543D303B2B31
:108B30004349505153454E443D313B45300D004172
:108B4000542B434F50533D300D0041540D004154C0
:108B5000480D0041542B435245473F3B2B4349505E
:108B60005354415455533B2B4353510D0041542B07
:0A8B70004950523D393630300D00F7
:068B7A0041424344454660
:108B80004748494A4B4C4D4E4F50515253545556FD
:108B90005758595A6162636465666768696A6B6CA5
:108BA0006D6E6F707172737475767778797A303113
:108BB00032333435363738392B2F007C2424247D4A
:108BC00072737475767778797A7B2424242424242C
:108BD000243E3F404142434445464748494A4B4C66
:108BE0004D4E4F505152535455565724242424244B
:108BF0002458595A5B5C5D5E5F60616263646566C0
:0C8C00006768696A6B6C6D6E6F707100C4
:048C0C00D9CFE6FFD7
:108C1000DACFE6FFE1CFD9FFE2CFDAFFFB0EDBCF01
:108C200000F0FC0EDBCF01F00001800E01141AE110
:108C3000FB0EDBCFE9FFFC0EDBCFEAFFEECFF3FF4D
:108C4000EDCFF4FFEE2A000EEF22F3CFE9FFF4CFD1
:108C5000EAFFFD0EDBCFEFFFEF50016AF36E01C0BC
:108C6000F4FF10D0FB0EDB50FE0806E1FD0EDBCF5B
:108C7000E6FF1BEC47F005D0FD0EDBCFE6FF03EC73
:108C800000F0E552E552E5CFDAFFE7CFD9FF120059
:108C900026502B02F3CF22F0F4CF23F02C02F35016
:108CA0002326000EF420246E26502D02F350242695
:108CB000000EF420256E26502E02F3502526275054
:108CC0002B02F3502326F4502422000E2522275095
:108CD0002C02F3502426F450252227502D02F35065
:108CE000252628502B02F3502426F4502522285004
:108CF0002C02F350252629502B02F3502526120072
:108D000092680E0EC16E8A0EC06E12008050020B69
:108D100001E0000C010CC26AC26AC280C282C2B207
:108D2000FED7C290C3CF28F0C4CF29F0B3EC34F003
:108D300027C004F028C005F029C006F02AC007F0BB
:108D40002C6A2D6A380E2E6E420E2F6EE3EC34F034
:108D500027C026F028C027F029C028F02AC029F013
:028D60001200FF
:0E8D6200256A246A236A226A200EE76ED890E2
:108D70002636273628362936223623362436253617
:108D80002B50225C2C5023582D5024582E502558FF
:108D900009E32B50225E2C50235A2D50245A2E507A
:0A8DA000255A262AE72EE4D7120018
:068DAA00256A246A100E88
:108DB000E76ED89028362936243625362D50245C87
:108DC0002E50255805E32D50245E2E50255A282A72
:068DD000E72EF0D71200AF
:0A8DD600F36AF46AFF0EE124E96E6F
:108DE000FF0EE220EA6EED6607D02F0EEF6404D08E
:0A8DF0003A0EEF6001D0F32A1200E2
:068DFA00000EF36E00EE16
:108E000000F00D0E01D81200EA6002D0EE6AFCD725
:0A8E1000F350E9601200EE6AFCD78F
:068E1A001CEE00F02CEE3E
:108E200000F0F86A219C1FEC45F007EC00F08FEC95
:068E300040F0FBD7120028
:0A8E3600FF0EE350ACBA04D0AF6A9F
:108E4000AB8EAC8A949CACA2FED7AD6EF36EF46A86
:028E500012000E
:0E8E5200256A080EE76ED890293625362E5078
:0E8E6000255C02E3256E292AE72EF7D71200C3
:028E6E003031A1
:0F8E7000323334353637383961626364656600F2
:018E7F0001F1
:108E800003010000000000000400000000000000DA
:108E90000000000000000000000000000000008151
:108EA0002D2D2D2D2D2D2D2D2D2D2D2D2D2D2D2DF2
:108EB0002D00000000000000000000000000000085
:108EC000000000D9C6DE16364A44FE00000000004D
:0C8ED000000000FFFFFFFFFF000000009B
:048EDC0062469A460A
:108EE000BE46F4460E4772478E4718486448B84855
:108EF000E6486449A849EE49164A644ABA4A124B00
:108F00002A4B404B564B6A4B804B024C284C4E4CE4
:028F10007C4C97
:0E8F1200000000000000000000000000000051
:108F20000000000000000000000000000000000041
:108F30000000000000000000000000000000000031
:058F400000000000002C
:0B8F450000000A000000000000000017
:108F50000000000000000000000000000000000011
:0E8F6000000000000000FF0000000000000004
:028F6E00800081
:108F700000000000000000000000000000000000F1
:108F800000000000000000000000000000000000E1
:108F900000000000000000000000000000000000D1
:0E8FA0000000000000000000000000000000C3
:028FAE000000C1
:028FB000004D72
:020000040030CA
:0100010002FC
:0100020000FD
:0100030017E5
:0100050000FA
:010006008178
:010008003FB8
:01000900C036
:01000A003FB6
:01000B00E014
:01000C003FB4
:01000D0040B2
:0200000400F00A
:100000004E4F50484F4E45000000000000000000D9
:1000100000000000000000000000000000000000E0
:100020004F564D530000000000000000000000008B
:1000300000000000000000000000000000000000C0
:100040004B00000000000000000000000000000065
:1000500000000000000000000000000000000000A0
:100060000000000000000000000000000000000090
:100070000000000000000000000000000000000080
:100080000000000000000000000000000000000070
:00000001FF
